:0300000002660B8A
:10660B00758E1190000078FF79FFE4F0A3D9FBD8C9
:0D661B00F778FFE4F6D8FD75817302666321
:10693F004401D240490FDB4401CE40C90FDB440173
:05694F00CA3C8EFA3580
:06472B009001B2121FA56F
:104731009001B6E0FCA3E0FDA3E0FEA3E0FFEF24BF
:1047410069FFEE3474FEED34FFFDEC34FFFCEC1236
:104751001B0F7BDF7A927986783D1218EB9001BAB4
:10476100121FA57B007A0079C078419001BAE0FC64
:10477100A3E0FDA3E0FEA3E0FF1219F4125E037BA8
:10478100007A0079C078411218EBC004C005C00658
:10479100C0077F977E7E7DD57C409001BAE0F8A36B
:1047A100E0F9A3E0FAA3E0FB1217FAD003D002D09C
:1047B10001D0001217F6C004C005C006C0077F92E1
:1047C1007E867DC07C419001B2E0F8A3E0F9A3E0D0
:1047D100FAA3E0FB1218EBA804A905AA06AB07D0BF
:1047E10007D006D005D0041217FA9001C2121FA5F6
:1047F1009001B6E0FCA3E0FDA3E0FEA3E0FFEF24FF
:1048010069FFEE3474FEED34FFFDEC34FFFCEC1275
:104811001B0F9001B2E0F8A3E0F9A3E0FAA3E0FBDB
:104821001217FA7B307AE67958783D1218EBA80412
:10483100A905AA06AB077F817E0E7DBA7C431217BC
:10484100F69001CAE0F8A3E0F9A3E0FAA3E0FB12B5
:1048510018EB9001BE121FA59001CEE0FCA3E0FD74
:10486100A3E0FEA3E0FF9001BEE0F8A3E0F9A3E01E
:10487100FAA3E0FB121A91602940279001BEE0FCE7
:10488100A3E0FDA3E0FEA3E0FF9001CEE0F8A3E0EA
:10489100F9A3E0FAA3E0FB1217F69001BE121FA5DF
:1048A10080B69001CEE0FCA3E0FDA3E0FEA3E0FF13
:1048B100121AFE9001BEE0F8A3E0F9A3E0FAA3E02A
:1048C100FB121A9150279001BEE0FCA3E0FDA3E08A
:1048D100FEA3E0FF9001CEE0F8A3E0F9A3E0FAA384
:1048E100E0FB1217FA9001BE121FA580B57F007E72
:1048F100007D007C009001BEE0F8A3E0F9A3E0FA9E
:10490100A3E0FB121A91604840469001D2E0FCA35B
:10491100E0FDA3E0FEA3E0FF9001BEE0F8A3E0F913
:10492100A3E0FAA3E0FB121A9150259001BEE0FC2E
:10493100A3E0FDA3E0FEA3E0FF9001CEE0F8A3E039
:10494100F9A3E0FAA3E0FB1217F69001BE121FA52E
:104951007F007E007D007C009001BEE0F8A3E0F9BD
:10496100A3E0FAA3E0FB121A91504B9001D2E0FCB4
:10497100A3E0FDA3E0FEA3E0FF121AFE9001BEE05A
:10498100F8A3E0F9A3E0FAA3E0FB121A9160274033
:10499100259001BEE0FCA3E0FDA3E0FEA3E0FF90B3
:1049A10001CEE0F8A3E0F9A3E0FAA3E0FB1217FAC5
:1049B1009001BE121FA59001BEE0FCA3E0FDA3E0A3
:1049C100FEA3E0FF1254FB7B247A0B79987839120D
:1049D10018EB9001C2E0F8A3E0F9A3E0FAA3E0FB31
:1049E1001217FA9001C6121FA57B007A0079C078D0
:1049F100419001C6E0FCA3E0FDA3E0FEA3E0FF12AD
:104A010019F4125E037B007A0079C078411218EB29
:104A1100A804A905AA06AB079001C6E0FCA3E0FD26
:094A2100A3E0FEA3E0FF1217F66A
:014A2A002269
:1068FD009001DD121FA59001DDE0FCA3E0FDA3E0FA
:10690D00FEA3E0FF125E03A804A905AA06AB07903B
:10691D0001DDE0FCA3E0FDA3E0FEA3E0FF1217F60E
:10692D009001CEE0F8A3E0F9A3E0FAA3E0FB121882
:02693D00EB224B
:060CC400900142121FA581
:100CCA00900142E0FCA3E0FDA3E0FEA3E0FFEF24D5
:100CDA0013FFEE342DFEED34FFFDEC34FFFCEC1275
:100CEA001B0F900146E0F8A3E0F9A3E0FAA3E0FBAA
:100CFA001217FA90014A121FA57F8D7EA67D147CD9
:100D0A003D90014AE0F8A3E0F9A3E0FAA3E0FB1260
:100D1A0018EB7B807AF279BF783E1217FA1268FDD7
:100D2A0090014E121FA57F477E857D167C3D90015E
:100D3A004AE0F8A3E0F9A3E0FAA3E0FB1218EB7B80
:100D4A00937AA77984783E1217FA1268FD900152B5
:100D5A00121FA57F217EB47D0A7C3D90014AE0F8EE
:100D6A00A3E0F9A3E0FAA3E0FB1218EB7BFF7ACD2C
:100D7A007953783F1217FA1268FD900156121FA58F
:100D8A007F4D7E6C7D337C3B90014AE0F8A3E0F90D
:100D9A00A3E0FAA3E0FB1218EB7B817A3D797E7817
:100DAA003F1217FA1268FD90015A121FA57F007EA2
:100DBA00007D007C40900156E0F8A3E0F9A3E0FA38
:100DCA00A3E0FB1218EBA804A905AA06AB07900139
:100DDA004EE0FCA3E0FDA3E0FEA3E0FF1217F6122B
:100DEA0054E57BF37A767914783F1218EBC004C085
:100DFA0005C006C00790014EE0FCA3E0FDA3E0FE9B
:100E0A00A3E0FF1254E57BE87AC1795178401218C1
:100E1A00EBA804A905AA06AB077FB17E737D717C96
:100E2A00421217F6D003D002D001D0001217F6C032
:100E3A0004C005C006C0077F007E007D007C40908C
:100E4A000156E0F8A3E0F9A3E0FAA3E0FB1218EBDD
:100E5A001254E57B0C7A5979ED783E1218EBA80406
:100E6A00A905AA06AB07D007D006D005D0041217E9
:100E7A00F690015E121FA57F007E007D007C4090E7
:100E8A000156E0F8A3E0F9A3E0FAA3E0FB1218EB9D
:100E9A00C004C005C006C0077F007E007D007C40FC
:100EAA0090014EE0F8A3E0F9A3E0FAA3E0FB1218E0
:100EBA00EBD003D002D001D0001217F61254E57B12
:100ECA00767A4F791E783D1218EBC004C005C00629
:100EDA00C0077F007E007D007C4090014EE0F8A3B1
:100EEA00E0F9A3E0FAA3E0FB1218EB1254E57B9CAD
:100EFA007A5A79B6783D1218EBA804A905AA06AB66
:100F0A000790015EE0FCA3E0FDA3E0FEA3E0FF1270
:100F1A0017F6A804A905AA06AB07D007D006D0057C
:100F2A00D0041217FAC004C005C006C0077F007EAD
:100F3A00007D007C40900156E0F8A3E0F9A3E0FAB6
:100F4A00A3E0FB1218EB90015AE0F8A3E0F9A3E042
:100F5A00FAA3E0FB1217F61254E57B687A96790435
:100F6A00783D1218EBA804A905AA06AB07D007D04A
:100F7A0006D005D0041217F690015E121FA57F0055
:100F8A007E007D007C40900156E0F8A3E0F9A3E0E2
:100F9A00FAA3E0FB1218EBA804A905AA06AB07906E
:100FAA00014EE0FCA3E0FDA3E0FEA3E0FF1217F66A
:100FBA0090015AE0F8A3E0F9A3E0FAA3E0FB1217C4
:100FCA00FA1254E57BD87A2A79C1783C1218EBC018
:100FDA0004C005C006C0077F007E007D007C4090EB
:100FEA000156E0F8A3E0F9A3E0FAA3E0FB1218EB3C
:100FFA00A804A905AA06AB0790014EE0FCA3E0FDF0
:10100A00A3E0FEA3E0FF1217F61254E57B727A33CF
:10101A0079DC783C1218EBA804A905AA06AB07905C
:10102A00015EE0FCA3E0FDA3E0FEA3E0FF1217F6D9
:10103A00D003D002D001D0001217F6C004C005C0F8
:10104A0006C00790015AE0F8A3E0F9A3E0FAA3E08A
:10105A00FB90014EE0FCA3E0FDA3E0FEA3E0FF123B
:10106A0017F61254E57B307A4C79A6783C1218EBC5
:10107A00A804A905AA06AB07D007D006D005D00454
:10108A001217F690015E121FA5900156E0FCA3E02C
:10109A00FDA3E0FEA3E0FF1254E57B0B7AD2798C24
:1010AA00783C1218EB90015EE0F8A3E0F9A3E0FAAD
:1010BA00A3E0FB1217FAC004C005C006C0079001DE
:1010CA005AE0FCA3E0FDA3E0FEA3E0FF90014EE09E
:1010DA00F8A3E0F9A3E0FAA3E0FB1217FA1254E529
:1010EA007B697AE37988783C1218EBA804A905AAE7
:1010FA0006AB07D007D006D005D0041217FA900124
:10110A005E121FA57F007E007D007C40900152E0A8
:10111A00F8A3E0F9A3E0FAA3E0FB1218EBA804A9EC
:10112A0005AA06AB0790014EE0FCA3E0FDA3E0FE92
:10113A00A3E0FF1217F61254E57BF97A4E794C7840
:10114A003C1218EBC004C005C006C00790015AE063
:10115A00FCA3E0FDA3E0FEA3E0FF1254E57BCD7AF9
:10116A00AF79E6783B1218EBA804A905AA06AB07E3
:10117A00D007D006D005D0041217FAC004C005C0A3
:10118A0006C0077F007E007D007C40900156E0F893
:10119A00A3E0F9A3E0FAA3E0FB1218EB90015AE0EE
:1011AA00F8A3E0F9A3E0FAA3E0FB1217FA1254E558
:1011BA007BBC7A5779AD783B1218EBA804A905AA2B
:1011CA0006AB07D007D006D005D0041217FAC00420
:1011DA00C005C006C0077F007E007D807C4090016C
:1011EA0056E0F8A3E0F9A3E0FAA3E0FB1218EBA893
:1011FA0004A905AA06AB0790014EE0FCA3E0FDA3F3
:10120A00E0FEA3E0FF1217F61254E57B4E7AB4799A
:10121A00AB783B1218EBA804A905AA06AB07D007BE
:10122A00D006D005D0041217F6900162121FA57FCE
:10123A00007E007D007C40900156E0F8A3E0F9A30F
:10124A00E0FAA3E0FB1218EBA804A905AA06AB076B
:10125A0090014EE0FCA3E0FDA3E0FEA3E0FF12171D
:10126A00F690015AE0F8A3E0F9A3E0FAA3E0FB1232
:10127A0017F61254E57BA97A6A7982783B1218EB41
:10128A00900162E0F8A3E0F9A3E0FAA3E0FB1217E9
:10129A00FAC004C005C006C0077F007E007D407CFE
:1012AA004090014EE0F8A3E0F9A3E0FAA3E0FB12B4
:1012BA0018EB1254E57B9C7ADC796F783B1218EBB9
:1012CA00A804A905AA06AB07D007D006D005D00402
:1012DA001217F6C004C005C006C0077F007E007D55
:1012EA00807C40900156E0F8A3E0F9A3E0FAA3E07D
:1012FA00FB1218EBC004C005C006C0077F007E00C1
:10130A007D007C4090014EE0F8A3E0F9A3E0FAA347
:10131A00E0FB1218EBD003D002D001D0001217F66E
:10132A001254E57BCA7A547941783B1218EBA80427
:10133A00A905AA06AB07D007D006D005D004121714
:10134A00F6900162121FA57F007E007D007C40900E
:10135A000156E0F8A3E0F9A3E0FAA3E0FB1218EBC8
:10136A00C004C005C006C0077F007E007D407C40E7
:10137A0090014EE0F8A3E0F9A3E0FAA3E0FB12180B
:10138A00EBD003D002D001D0001217F61254E57B3D
:10139A00457A2F7923783B1218EBC004C005C006A2
:1013AA00C00790015AE0FCA3E0FDA3E0FEA3E0FF22
:1013BA00900156E0F8A3E0F9A3E0FAA3E0FB1217C4
:1013CA00FA1254E57B147A5C792C783B1218EBA854
:1013DA0004A905AA06AB07900162E0FCA3E0FDA3FD
:1013EA00E0FEA3E0FF1217F6A804A905AA06AB07B8
:1013FA00D007D006D005D0041217FAC004C005C021
:10140A0006C0077F007E007D007C40900156E0F810
:10141A00A3E0F9A3E0FAA3E0FB1218EB90014EE077
:10142A00F8A3E0F9A3E0FAA3E0FB1217FA90015A35
:10143A00E0F8A3E0F9A3E0FAA3E0FB1217F61254CE
:10144A00E57BA67AD57910783B1218EBA804A90592
:10145A00AA06AB07D007D006D005D0041217F6C0EB
:10146A0004C005C006C0077F007E007D007C409056
:10147A000156E0F8A3E0F9A3E0FAA3E0FB1218EBA7
:10148A00C004C005C006C0077F007E007D007C4006
:10149A00900152E0F8A3E0F9A3E0FAA3E0FB1218E6
:1014AA00EBD003D002D001D0001217F61254E57B1C
:1014BA00B37A7B79F2783A1218EBA804A905AA063E
:1014CA00AB07D007D006D005D0041217FA900162F4
:1014DA00121FA57F007E007D007C40900152E0F83B
:1014EA00A3E0F9A3E0FAA3E0FB1218EB90014EE0A7
:1014FA00F8A3E0F9A3E0FAA3E0FB1217FAC004C0CC
:10150A0005C006C0077F007E007D007C4090015622
:10151A00E0F8A3E0F9A3E0FAA3E0FB1218EBA804B1
:10152A00A905AA06AB07D007D006D005D004121722
:10153A00F61254E57B047AAD79C0783A1218EBC0FA
:10154A0004C005C006C0077F007E007D007C409075
:10155A00015AE0F8A3E0F9A3E0FAA3E0FB1218EBC2
:10156A00C004C005C006C0077F007E007D007C4025
:10157A00900156E0F8A3E0F9A3E0FAA3E0FB121801
:10158A00EBD003D002D001D0001217F61254E57B3B
:10159A00A37A0679D378BA1218EBA804A905AA0681
:1015AA00AB07D007D006D005D0041217FAC004C082
:1015BA0005C006C0077F007E007D807C40900156F2
:1015CA00E0F8A3E0F9A3E0FAA3E0FB1218EB125447
:1015DA00E57B4B7A1F79BA783A1218EBA804A90569
:1015EA00AA06AB07D007D006D005D0041217F6C05A
:1015FA0004C005C006C0077F007E007D007C4090C5
:10160A000156E0F8A3E0F9A3E0FAA3E0FB1218EB15
:10161A00C004C005C006C0077F007E007D007C4074
:10162A0090014EE0F8A3E0F9A3E0FAA3E0FB121858
:10163A00EBD003D002D001D0001217F690015AE085
:10164A00F8A3E0F9A3E0FAA3E0FB1217FA1254E5B3
:10165A007BA97A3079B6783A1218EBA804A905AAB8
:10166A0006AB07D007D006D005D0041217FA9001AE
:10167A0066121FA57F007E007D807C40900156E0A7
:10168A00F8A3E0F9A3E0FAA3E0FB1218EBA804A977
:10169A0005AA06AB0790014EE0FCA3E0FDA3E0FE1D
:1016AA00A3E0FF1217F690015AE0F8A3E0F9A3E0CD
:1016BA00FAA3E0FB1217FA1254E57B3B7AAA799A4D
:1016CA00783A1218EBA804A905AA06AB0790016696
:1016DA00E0FCA3E0FDA3E0FEA3E0FF1217F6C004BE
:1016EA00C005C006C0077F007E007D007C409001D7
:1016FA0056E0F8A3E0F9A3E0FAA3E0FB1218EBC066
:10170A0004C005C006C0077F007E007D007C4090B3
:10171A00014EE0F8A3E0F9A3E0FAA3E0FB1218EB0C
:10172A00A804A905AA06AB07D007D006D005D0049D
:10173A001217FA1254E57B247A0B7998783A121820
:10174A00EBA804A905AA06AB07D007D006D005D096
:10175A00041217F6C004C005C006C0077F007E0049
:10176A007D007C4090014EE0F8A3E0F9A3E0FAA3E3
:10177A00E0FB1218EB90015AE0F8A3E0F9A3E0FAB3
:10178A00A3E0FB1217F61254E57BE07A2D799078E4
:10179A003A1218EBA804A905AA06AB07D007D00687
:1017AA00D005D0041217F6900166121FA5900162A7
:1017BA00E0FCA3E0FDA3E0FEA3E0FF90015EE0F8F9
:1017CA00A3E0F9A3E0FAA3E0FB1217FA900166E09E
:1017DA00F8A3E0F9A3E0FAA3E0FB1217FA7B487A30
:0817EA005179C778451218EB94
:0117F20022D4
:0B2A1C00900108EBF0A3EAF0A3E9F042
:102A270090010EE0FCA3E0FDA3E0FEA3E0FFEC12A3
:102A37001B0F7B007A81798878C61217FA900112EA
:102A4700E0F8A3E0F9A3E0FAA3E0FB1217FA90017C
:102A570016121FA57F0A7EEB7D157C3D900116E0BF
:102A6700F8A3E0F9A3E0FAA3E0FB1218EB7B7F7A67
:102A77004F7940783F1217FA1268FD90011A121F1A
:102A8700A57F8C7EA67D147C3D900116E0F8A3E01F
:102A9700F9A3E0FAA3E0FB1218EB7B367A907952A0
:102AA700783F1217FA1268FD90011E121FA57F4D7D
:102AB7007E6C7D337C3B900116E0F8A3E0F9A3E040
:102AC700FAA3E0FB1218EB7B857AEA797E783F124E
:102AD70017FA1268FD900122121FA57F217EB47D8F
:102AE7000A7C3D900116E0F8A3E0F9A3E0FAA3E021
:102AF700FB1218EB7BD37A697979783F1217FA12B0
:102B070068FD900126121FA57F477E857D167C3DB7
:102B1700900116E0F8A3E0F9A3E0FAA3E0FB12188E
:102B2700EB7B9F7A027900783D1217FA1268FD90C5
:102B3700012A121FA57F007E007D007C40900126A0
:102B4700E0F8A3E0F9A3E0FAA3E0FB1218EB1254B4
:102B5700FB7BB07A727928783F1218EBC004C00566
:102B6700C006C00790011EE0FCA3E0FDA3E0FEA3A2
:102B7700E0FF1254FB7B7D7A3F79C978401218EB4E
:102B8700A804A905AA06AB07D007D006D005D0042C
:102B97001217FAC004C005C006C0077F007E007D7B
:102BA700007C40900126E0F8A3E0F9A3E0FAA3E057
:102BB700FB1218EBA804A905AA06AB0790011EE0B3
:102BC700FCA3E0FDA3E0FEA3E0FF1217F61254FBFF
:102BD7007B6F7A1279A3783F1218EBA804A905AA8C
:102BE70006AB07D007D006D005D0041217F6C004ED
:102BF700C005C006C007900122E0FCA3E0FDA3E0EA
:102C0700FEA3E0FF1254FB7BC97A76793E783E1229
:102C170018EBA804A905AA06AB07D007D006D0056C
:102C2700D0041217F69001CAE0F8A3E0F9A3E0FA7E
:102C3700A3E0FB1218EB90011AE0F8A3E0F9A3E078
:102C4700FAA3E0FB1217FA90012E121FA590012E8E
:102C5700E0FCA3E0FDA3E0FEA3E0FFC004C005C0C5
:102C670006C0077F007E007D007C4090012AE0F8C7
:102C7700A3E0F9A3E0FAA3E0FB1218EB1254FB7BE5
:102C8700D57A7879E9783D1218EBC004C005C006FB
:102C9700C0077F007E007D007C4090011EE0F8A306
:102CA700E0F9A3E0FAA3E0FB1218EB1254FB7BD187
:102CB7007A22795B783E1218EBD003D002D001D08C
:102CC700001217F6C004C005C006C0077F007E00CB
:102CD7007D007C40900126E0F8A3E0F9A3E0FAA389
:102CE700E0FB1218EBC004C005C006C0077F007EDA
:102CF700007D007C4090011EE0F8A3E0F9A3E0FA14
:102D0700A3E0FB1218EBD003D002D001D0001217BA
:102D1700F61254FB7BFC7AA97971783D1218EBA85F
:102D270004A905AA06AB07D007D006D005D0041220
:102D370017F6C004C005C006C0077F007E007D00EF
:102D47007C40900126E0F8A3E0F9A3E0FAA3E0FBBA
:102D57001218EBC004C005C006C007900122E0FCB2
:102D6700A3E0FDA3E0FEA3E0FF90011EE0F8A3E0CF
:102D7700F9A3E0FAA3E0FB1217FAD003D002D001BF
:102D8700D0001217F61254FB7BD57A787969783D13
:102D97001218EBA804A905AA06AB07D007D006D0DE
:102DA70005D0041217F69001CAE0F8A3E0F9A3E0F2
:102DB700FAA3E0FB1218EBA804A905AA06AB07D0F3
:102DC70007D006D005D0041217FA90012E121FA5BE
:102DD7007F007E007D007C40900126E0F8A3E0F9AB
:102DE700A3E0FAA3E0FB1218EB1254FB7BE37AC7CC
:102DF7007928783F1218EBC004C005C006C00790B9
:102E0700011EE0FCA3E0FDA3E0FEA3E0FF1254FBDC
:102E17007B9E7A5E79C778401218EBA804A905AAA9
:102E270006AB07D007D006D005D0041217FAC004A6
:102E3700C005C006C0077F007E007D007C40900172
:102E470026E0F8A3E0F9A3E0FAA3E0FB1218EBA849
:102E570004A905AA06AB0790011EE0FCA3E0FDA3A9
:102E6700E0FEA3E0FF1217F61254FB7BE57AD07958
:102E7700A2783F1218EBA804A905AA06AB07D0074A
:102E8700D006D005D0041217F69001CAE0F8A3E0E7
:102E9700F9A3E0FAA3E0FB1218EB90012AE0F8A3EC
:102EA700E0F9A3E0FAA3E0FB1217FA900132121F30
:102EB700A57F007E007D007C40900126E0F8A3E01E
:102EC700F9A3E0FAA3E0FB1218EBA804A905AA06E8
:102ED700AB0790012AE0FCA3E0FDA3E0FEA3E0FF1F
:102EE7001217F61254FB7B067A817915783E121871
:102EF700EBC004C005C006C007900132E0FCA3E0A8
:102F0700FDA3E0FEA3E0FF1254FB7BA67A9B79A406
:102F170078401218EBD003D002D001D0001217F678
:102F27009001CAE0F8A3E0F9A3E0FAA3E0FB1218C6
:102F3700EB900136121FA590012EE0FCA3E0FDA344
:102F4700E0FEA3E0FF1254FBC004C005C006C007A3
:102F5700900136E0FCA3E0FDA3E0FEA3E0FF1254DE
:102F6700E5A804A905AA06AB07D007D006D005D067
:102F7700041218EB7B327AAF79CB783E1218EBC08C
:102F870004C005C006C007900136E0FCA3E0FDA31E
:102F9700E0FEA3E0FF1254FB7BDB7ADE796A783F21
:102FA7001218EBA804A905AA06AB07D007D006D0CC
:102FB70005D0041217FA90010BE0FBA3E0FAA3E097
:102FC700F9121F3390010BE0FBA3E0FAA3E0F9121B
:102FD7001F1390010BE0FBA3E0FAA3E0F9121F8592
:102FE7001218EBA804A905AA06AB077F007E007D8F
:102FF700807C3F1217F612641B9000D0121FA59019
:10300700010BE0FBA3E0FAA3E0F9121F131266A875
:1030170090010BE0FBA3E0FAA3E0F9121F33900144
:103027002EE0FCA3E0FDA3E0FEA3E0FF1254E5C001
:1030370004C005C006C007900136E0FCA3E0FDA36D
:10304700E0FEA3E0FF1254E5A804A905AA06AB0712
:10305700D007D006D005D0041218EBC004C005C0B5
:1030670006C00790010BE0FBA3E0FAA3E0F9121FEB
:10307700131254E5A804A905AA06AB07D007D00682
:10308700D005D0041219F490013A121FA590012E11
:10309700E0FCA3E0FDA3E0FEA3E0FF1254FBC004A5
:1030A700C005C006C007900136E0FCA3E0FDA3E021
:1030B700FEA3E0FF1254E5A804A905AA06AB07D0B2
:1030C70007D006D005D0041218EB7BDB7ADE796ACD
:1030D700783F1218EBC004C005C006C00790013640
:1030E700E0FCA3E0FDA3E0FEA3E0FF1254FB7B326C
:1030F7007AAF79CB783E1218EBA804A905AA06ABDC
:1031070007D007D006D005D0041217F6C004C005B3
:10311700C006C00790010BE0FBA3E0FAA3E0F91299
:103127001F131254E5A804A905AA06AB07D007D0B8
:1031370006D005D0041219F490013E121FA5900184
:103147003EE0FCA3E0FDA3E0FEA3E0FFC004C00552
:10315700C006C00790013AE0FCA3E0FDA3E0FEA390
:10316700E0FF9000D0121FA5D007D006D005D004ED
:103177001266A8900108E0FBA3E0FAA3E0F9121F8A
:1031870033900108E0FBA3E0FAA3E0F9121F137BD9
:10319700007A0079007800121A916030402E900171
:1031A70008E0FBA3E0FAA3E0F9C003C002C00112E4
:1031B7001F139001CEE0F8A3E0F9A3E0FAA3E0FB28
:1031C7001217FAD001D002D003121F33900108E082
:1031D700FBA3E0FAA3E0F9121F139001CEE0F8A3D6
:1031E700E0F9A3E0FAA3E0FB121A91502E90010830
:1031F700E0FBA3E0FAA3E0F9C003C002C001121F7D
:10320700139001CEE0F8A3E0F9A3E0FAA3E0FB12E4
:0B32170017F6D001D002D003121F33C5
:013222002289
:0B400800900190EBF0A3EAF0A3E9F0B8
:10401300900196E0FCA3E0FDA3E0FEA3E0FFEC1219
:104023001B0F7B007A81798878C61217FA90019A60
:10403300E0F8A3E0F9A3E0FAA3E0FB1217FA7B0090
:104043007AAD790E78471219F490019E121FA57F5D
:10405300A67EFE7DC77C4290019EE0F8A3E0F9A313
:10406300E0FAA3E0FB1218EB7B917AEA797E783FC2
:104073001217FA1268FD9001A2121FA57F117E2369
:104083007D5F7C3790019EE0F8A3E0F9A3E0FAA3FB
:10409300E0FB1218EBA804A905AA06AB077F507E24
:1040A300AC7DAE7C3B1217F61268FDC004C005C0A0
:1040B30006C0079001A2E0FCA3E0FDA3E0FEA3E09D
:1040C300FF1254FBA804A905AA06AB07D007D00624
:1040D300D005D0041218EBC004C005C006C0077F8A
:1040E300187E017DC87C4290019EE0F8A3E0F9A30D
:1040F300E0FAA3E0FB1218EB7B327AE47946783FCF
:104103001217FA1268FDA804A905AA06AB07D0077F
:10411300D006D005D0041217FAC004C005C006C0EB
:10412300077F007E007D007C409001A2E0F8A3E0C1
:10413300F9A3E0FAA3E0FB1218EB1254FB7B0C7A11
:1041430034796978381218EBA804A905AA06AB07D5
:10415300D007D006D005D0041217FA9001A6121F7B
:10416300A57F147E6A7D177C3890019EE0F8A3E05A
:10417300F9A3E0FAA3E0FB1218EBA804A905AA0629
:10418300AB077F6D7E6A7D857C3D1217F61268FD55
:104193009001AA121FA59001A6E0FCA3E0FDA3E0F5
:1041A300FEA3E0FF125537C004C005C006C0079048
:1041B30001AAE0FCA3E0FDA3E0FEA3E0FF1254E5A7
:1041C300A804A905AA06AB07D007D006D005D004DA
:1041D3001218EB1259EC900190E0FBA3E0FAA3E074
:1041E300F9121F339001CEE0F8A3E0F9A3E0FAA39C
:1041F300E0FB9001A6E0FCA3E0FDA3E0FEA3E0FF4B
:104203001219F4125E039001CEE0F8A3E0F9A3E0E3
:10421300FAA3E0FB1218EBA804A905AA06AB0790C2
:1042230001A6E0FCA3E0FDA3E0FEA3E0FF1217F666
:104233009001AE121FA57F007E007DC07C3F9001E0
:10424300D2E0F8A3E0F9A3E0FAA3E0FB1218EB90A5
:1042530001AEE0F8A3E0F9A3E0FAA3E0FB121A91A0
:10426300505A7F007E007D007C3F9001D2E0F8A38E
:10427300E0F9A3E0FAA3E0FB1218EB9001AEE0F83B
:10428300A3E0F9A3E0FAA3E0FB121A91402E9001F8
:1042930090E0FBA3E0FAA3E0F9C003C002C001125F
:1042A3001F139001D2E0F8A3E0F9A3E0FAA3E0FB27
:1042B3001217FAD001D002D003121F33900190E0FD
:1042C300FBA3E0FAA3E0F9C003C002C001121F136D
:1042D300C004C005C006C007900190E0FBA3E0FA4C
:1042E300A3E0F9121F139001CEE0F8A3E0F9A3E0D5
:1042F300FAA3E0FB1219F4125E039001CEE0F8A3D7
:10430300E0F9A3E0FAA3E0FB1218EBA804A905AABD
:1043130006AB07D007D006D005D0041217F6D0019C
:10432300D002D003121F339001A6E0FCA3E0FDA34B
:10433300E0FEA3E0FF1254FBC004C005C006C007A3
:104343009001AAE0FCA3E0FDA3E0FEA3E0FF12546A
:10435300FBA804A905AA06AB07D007D006D005D051
:10436300041218EB900193E0FBA3E0FAA3E0F91227
:104373001F33900193E0FBA3E0FAA3E0F9121F13AC
:10438300900193E0FBA3E0FAA3E0F9121F85121852
:10439300EBA804A905AA06AB077F007E007D807CFD
:1043A3003F1217F612641B9000D0121FA5900193C1
:1043B300E0FBA3E0FAA3E0F9121F131266A8900131
:0C43C30093E0FBA3E0FAA3E0F9121F3323
:0143CF0022CB
:0B32230090016AEBF0A3EAF0A3E9F0D1
:10322E007F927E0A7D867C3E900170E0F8A3E0F9E5
:10323E00A3E0FAA3E0FB1218EB900174E0F8A3E010
:10324E00F9A3E0FAA3E0FB1217F690017C121FA57A
:10325E007F007E007D007C0090017CE0F8A3E0F909
:10326E00A3E0FAA3E0FB121A91502790017CE0FC38
:10327E00A3E0FDA3E0FEA3E0FF9001CEE0F8A3E003
:10328E00F9A3E0FAA3E0FB1217FA90017C121FA536
:10329E0080489001CEE0FCA3E0FDA3E0FEA3E0FF9A
:1032AE0090017CE0F8A3E0F9A3E0FAA3E0FB121A88
:1032BE00916027402590017CE0FCA3E0FDA3E0FE99
:1032CE00A3E0FF9001CEE0F8A3E0F9A3E0FAA3E0BB
:1032DE00FB1217F690017C121FA590017CE0F8A35B
:1032EE00E0F9A3E0FAA3E0FB90001EE0FCA3E0FDF2
:1032FE00A3E0FEA3E0FF1217F6900016121FA59092
:10330E000016E0FCA3E0FDA3E0FEA3E0FF1254E5EF
:10331E00C004C005C006C00790001AE0FCA3E0FD83
:10332E00A3E0FEA3E0FF1254E5A804A905AA06AB8C
:10333E0007D007D006D005D0041218EBC004C00584
:10334E00C006C007900178E0FCA3E0FDA3E0FEA359
:10335E00E0FF1254E5A804A905AA06AB07D007D0D2
:10336E0006D005D0041218EBC004C005C006C00775
:10337E0090001AE0FCA3E0FDA3E0FEA3E0FF1254D0
:10338E00FBC004C005C006C007900178E0FCA3E0B6
:10339E00FDA3E0FEA3E0FF1254FBA804A905AA06B4
:1033AE00AB07D007D006D005D0041218EBA804A99D
:1033BE0005AA06AB07D007D006D005D0041217FA1F
:1033CE00900180121FA5900180E0FCA3E0FDA3E018
:1033DE00FEA3E0FF900180E0F8A3E0F9A3E0FAA3DA
:1033EE00E0FB1218EBA804A905AA06AB077F007E26
:1033FE00007D807C3F1217F612641B900184121F11
:10340E00A5900180E0FCA3E0FDA3E0FEA3E0FFC0D9
:10341E0004C005C006C007900184E0FCA3E0FDA334
:10342E00E0FEA3E0FF9000D0121FA5D007D006D07B
:10343E0005D0041266A890016DE0FBA3E0FAA3E0AC
:10344E00F9121F3390016DE0FBA3E0FAA3E0F9122D
:10345E001F131254E5C004C005C006C00790016DCD
:10346E00E0FBA3E0FAA3E0F9121F131254FBD00302
:10347E00D002D001D0001219F4C004C005C006C09D
:10348E000790001AE0FCA3E0FDA3E0FEA3E0FF120C
:10349E0054E5C004C005C006C00790001AE0FCA3A6
:1034AE00E0FDA3E0FEA3E0FF1254FBD003D002D058
:1034BE0001D0001219F4A804A905AA06AB07D0077B
:1034CE00D006D005D0041218EBC004C005C006C04B
:1034DE000790016DE0FBA3E0FAA3E0F9121F1312AF
:1034EE0054E5C004C005C006C00790001AE0FCA356
:1034FE00E0FDA3E0FEA3E0FF1254E5A804A905AA8F
:10350E0006AB07D007D006D005D0041218EBC004C6
:10351E00C005C006C007900178E0FCA3E0FDA3E063
:10352E00FEA3E0FF1254FBD003D002D001D0001254
:10353E0019F4D003D002D001D0001217F690018CEE
:10354E00121FA5900178E0FCA3E0FDA3E0FEA3E02E
:10355E00FF1254E5C004C005C006C00790001AE073
:10356E00FCA3E0FDA3E0FEA3E0FF1254E5A804A92E
:10357E0005AA06AB07D007D006D005D0041218EB6B
:10358E00C004C005C006C007900016E0FCA3E0FD15
:10359E00A3E0FEA3E0FF1254E5A804A905AA06AB1A
:1035AE0007D007D006D005D0041218EBC004C00512
:1035BE00C006C007900178E0FCA3E0FDA3E0FEA3E7
:1035CE00E0FF1254FBC004C005C006C00790001AED
:1035DE00E0FCA3E0FDA3E0FEA3E0FF1254FBA80471
:1035EE00A905AA06AB07D007D006D005D00412183D
:1035FE00EBA804A905AA06AB07D007D006D005D0C4
:10360E00041217FA900188121FA5900178E0FCA30E
:10361E00E0FDA3E0FEA3E0FF1254E5C004C005C028
:10362E0006C007900016E0FCA3E0FDA3E0FEA3E0B9
:10363E00FF1254FBA804A905AA06AB07D007D006B3
:10364E00D005D0041218EBC004C005C006C0079008
:10365E000188E0FCA3E0FDA3E0FEA3E0FF9001885B
:10366E00E0F8A3E0F9A3E0FAA3E0FB1218EBA8043C
:10367E00A905AA06AB077F007E007D807C3F12174E
:10368E00F612641BA804A905AA06AB07D007D0063C
:10369E00D005D0041219F4900188121FA59001884C
:1036AE00E0FCA3E0FDA3E0FEA3E0FFC004C005C064
:1036BE0006C00790018CE0FCA3E0FDA3E0FEA3E0B2
:1036CE00FF9000D0121FA5D007D006D005D004124F
:1036DE0066A890016AE0FBA3E0FAA3E0F9121F339B
:1036EE0090016AE0FBA3E0FAA3E0F9121F137B003E
:1036FE007A0079007800121A916030402E90016A9B
:10370E00E0FBA3E0FAA3E0F9C003C002C001121F60
:10371E00139001CEE0F8A3E0F9A3E0FAA3E0FB12C8
:0B372E0017FAD001D002D003121F33A5
:01373900226D
:10636B00323B171C0205006400640001000007A308
:10637B00008703840064070803840682056900070D
:10638B0000020009003B003B0017001C000C0063DF
:10639B0000C700C70002000A0E0F03840E0F038410
:1063AB000E0F07080E0F070800070005000E000070
:1063BB0000000000000100010000000100010000CE
:1063CB0000000000000000000000000000000000C2
:1063DB0000000000000000000000000300000003AC
:1063EB00000200030002000300030002000300028E
:1063FB000003000000030001000300020003000281
:0C640B0000030003000200030002000375
:06695400C112C114C113C1
:1067D6009000107432F0900011743BF09000127427
:1067E60017F0900013741CF09000147402F09000DF
:1067F600157405F0124CF4756D00756E00D3E56ED8
:10680600940EE56D64809480503CE56E25E0FFE5CE
:106816006D33FE74712FF58274633EF583E493FC49
:10682600740193FDE56E25E0FFE56D33FE74222FBE
:10683600F58274003EF583ECF0A3EDF0056EE56E8F
:0A6846007002056D80B7124DF822B4
:103BBD0090003FE0F568D3E56864809482400BC3C4
:103BCD00E568648094865002C212E5A064FFFFEFA1
:103BDD005407F56AE56A6006C29CC2988002D29CC1
:103BED00E56A5406FFEF6027056CE56CD3940A4037
:103BFD000F75690AC3E568648094865003756C0A75
:103C0D00E56CD39414400E756964756C148006755B
:103C1D006C00756901AF68EF3395E0FEEF25E0FFAD
:103C2D00EE33FE74B92FF58274633EF583E493F59C
:103C3D0066740193F567AF68EF3395E0FEEF25E00D
:103C4D00FFEE33FE748F2FF58274633EF583E4939C
:103C5D00F564740193F565E5686403706B90001568
:103C6D00E0FFEF75F004121DCDAFF0EF602E900068
:103C7D0014E0FFEF3395E0FEEF25E0FFEE33FE7429
:103C8D00E32FF58274633EF583E493FE740193FF95
:103C9D00EF2565F565EE3564F564802C900014E034
:103CAD00FFEF3395E0FEEF25E0FFEE33FE74FD2FC1
:103CBD00F58274633EF583E493FE740193FFEF2563
:103CCD0065F565EE3564F564E56AB401109000287C
:103CDD00E0FEA3E0FFEF4E7004056B8003756B00F3
:103CED00E56BC394144008756B00A212B39212D306
:103CFD00E56A648094815003023FACC3E56864803B
:103D0D0094864003023DD2124D49E56A6404705514
:103D1D00AF68EF3395E0FE74102FF58274003EF519
:103D2D0083E02569F0AF68EF3395E0FE74102FF551
:103D3D008274003EF583E0FFEF3395E0FED3EF95FF
:103D4D0065E5646480F8EE6480984016AF67AE68F0
:103D5D00EEFD3395E0FC74102DF58274003CF58377
:103D6D00EFF0124CF4E56A6402705AAF68EF3395C8
:103D7D00E0FE74102FF58274003EF583E0FFC3EF73
:103D8D009569FFEFF0AF68EF3395E0FE74102FF5F6
:103D9D008274003EF583E0FFEF3395E0FEC3EF95AF
:103DAD0067E5666480F8EE6480985016AF65AE687E
:103DBD00EEFD3395E0FC74102DF58274003CF58317
:103DCD00EFF0124CF4C3E568648094865003023E14
:103DDD00EE74FA2568F568E56A64047072AF69EFF0
:103DED00FD7C00AF68EF3395E0FEEF25E0FFEE338D
:103DFD00FE74222FF58274003EF583EC8DF0121EB9
:103E0D008FAF68EF3395E0FEEF25E0FFEE33FE74E4
:103E1D00222FF58274003EF583E0FEA3E0FFD3EF81
:103E2D009565E5646480F8EE648098401FAF68EF97
:103E3D003395E0FEEF25E0FFEE33FE74222FF58281
:103E4D0074003EF583E566F0A3E567F0124DF8E5E5
:103E5D006A64026003023EE8AF68EF3395E0FEEF5F
:103E6D0025E0FFEE33FE74222FF58274003EF583BC
:103E7D00C083C082E0FEA3E0FFAD697C00C3EF9D6F
:103E8D00FFEE9CFED082D083EEF0A3EFF0AF68EF93
:103E9D003395E0FEEF25E0FFEE33FE74222FF58221
:103EAD0074003EF583E0FEA3E0FFC3EF9567E56682
:103EBD006480F8EE648098501FAF68EF3395E0FE94
:103ECD00EF25E0FFEE33FE74222FF58274003EF5F0
:103EDD0083E564F0A3E565F0124DF874062568F5E9
:103EED0068900028E0FEA3E0FFEF4E705CE56AB439
:103EFD0005263014230568AF68D3EF648094934092
:103F0D0003756800C214AF68EF3395E0FE90003E74
:103F1D00EEF0A3EFF0124DF8E56A64036003023F83
:103F2D00AC30147B1568AF68C3EF64809480500388
:103F3D00756813C214AF68EF3395E0FE90003EEE46
:103F4D00F0A3EFF0124DF88056E56AB40526301453
:103F5D00230568AF68D3EF648094924003756800C1
:103F6D00C214AF68EF3395E0FE90003EEEF0A3EF84
:103F7D00F0124DF8E56AB403263014231568AF68C6
:103F8D00C3EF648094805003756812C214AF68EF5C
:103F9D003395E0FE90003EEEF0A3EFF0124DF8E504
:103FAD006AB40102D214E56A5406FFEF6010900066
:103FBD003EE0FEA3E0FFEF64094E7002C2179001D0
:103FCD00E9E0FEA3E0FF900028E0FCA3E0FDED6F2B
:103FDD007002EC6E6002C217900028E0FEA3E0FFB5
:103FED009001E9EEF0A3EFF030A302D21320A30A63
:0A3FFD00301307C213A217B3921786
:014007002296
:104CF400124E4174A0124E597402124E5990001073
:104D04007C03E0124E1A124E59A3DCF6E0124E1A3E
:104D1400F5F0A3A3E0030354C045F0124E599000EC
:104D240014E0124E1A124E59C2B4124E34124E41AD
:104D340074A0124E5974F0124E59A3E0124E59C287
:104D4400B4124E3422124E4174A0124E59740212FF
:104D54004E59124E4174A004124E59900010124E36
:104D64007E124E22F0A3124E91124E7E124E22F06B
:104D7400A3124E91124E7E124E22F0A3124E9112A5
:104D84004E7EFB543F124E22F0A3124E91124E7EE1
:104D9400FA541F124E22F0EB23235403FD124E8BC0
:104DA400C2B4124E34124E4174A0124E5974F01211
:104DB4004E59124E4174A004124E59124E7EFB54A9
:104DC40003C39D2405838007030201000302012B12
:104DD400A3F0F5F0124E8BC2B4124E34124E41744D
:104DE400A0124E5974F0124E59E5F0124E59C2B445
:104DF400124E34227AA07B807C1E900022124ED167
:104E0400227AA07B80124E99ED900022F07AA0A322
:104E14007C1D124F062275F00A84C425F022C0E0DE
:0D4E2400C4540F75F00AA4F5F0D0E0540F4F
:104E310025F02200D2B5000000D2B400000000220B
:104E4100124E34C2B4000000C2B500000022D2B537
:104E5100000000C2B50000227E083392B4124E4F0A
:104E6100DEF833D2B40000A2B450040000A2B412A0
:104E71004E4F400122C2B40000124E34227E08A2DD
:104E8100B43300124E4FDEF7C322D2B4124E4F227A
:104E9100C2B4124E4FD2B422124E41EA124E59EB15
:104EA100124E59124E41EA04124E59124E7EFD1213
:104EB1004E8BC2B4124E3422124E41EA124E59EBBD
:104EC100124E59E6124E5908DCF9C2B4124E342280
:104ED100124E41EA124E59EB124E59E0124E59A3AD
:104EE100DCF9C2B4124E3422124E41EA04124E5978
:104EF1008003124E91124E7EF608DCF6124E8BC2E2
:104F0100B4124E3422124E41EA04124E5980031259
:104F11004E91124E7EF0A3DCF6124E8BC2B4124EAD
:024F2100342238
:104A2B00202020202531642E253032642025303281
:104A3B0062753A25303262753A2530326275202024
:104A4B00202000202020202532642E2531642025B3
:104A5B00303262753A25303262753A2530326275E2
:104A6B002020202000253033642E25316420202582
:104A7B003032642E25316420415A2F454C31202091
:104A8B002000253033642E253164202025303264FC
:104A9B002E25316420415A2F454C322020200025F1
:104AAB003033642E2531642020253032642E25319D
:104ABB00642052412F44454320202000253033648D
:104ACB002E2531645720253032642E2531644E203B
:104ADB004C4F2F4C41202020002530326275202076
:104AEB00202530326275202025303262753A253010
:104AFB003262753A25303262752020202000253035
:104B0B00352E31662020253032642E25316420204D
:104B1B00202020202025303264202000202B25301F
:104B2B0031642E2530316420202B253031642E2525
:104B3B0030316420434F52202053545020002530F5
:104B4B0033642E2531642020253032642E253164C8
:104B5B0020414E5420202531642E25316420002025
:104B6B002020204F20452035204A2046204C202055
:104B7B00202020002020202020202020454D4520D3
:104B8B0020202020202020200020416E74656E6E96
:104B9B006120436F6E74726F6C6C65722000202005
:104BAB0020202020207620352E3120202020202070
:104BBB002020002020204A414E4645424D41524183
:104BCB0050524D41594A554E4A554C415547534504
:104BDB00504F43544E4F56444543004D4F4F4E207C
:104BEB002053554E20202043415353494F4359479F
:104BFB004E55535341474954545441555255534CB8
:104C0B00454F20202041515541522E52412F4445B2
:104C1B0043415A2F454C32415A2F454C3100326D8E
:104C2B003A37303A32333A31333A36636D313047B3
:104C3B0000205353492031306269742837323029B0
:104C4B0020202020202053534931316269742831B0
:104C5B003830302920202020202053534931326214
:104C6B0069742833363030292020202020205353DC
:104C7B00495F67726179283430393629202020202A
:104C8B00202041322D532D53203132206269742064
:104C9B0020202020204D414232355F313062697433
:104CAB003130323420202020204D414232355F31CB
:104CBB00316269743230343820202020204D41423B
:104CCB0032355F313262697434303936202020201E
:104CDB0020000F0C09010306171D664C030903097D
:094CEB000309030956010102044A
:10002E00E56A64016003125BB4200D0302060CC284
:10003E000D30120C900028E0FEA3E0FFEF4E601191
:10004E0090003EE0FEA3E0FFEF64134E600302015A
:10005E00E390003CE0FEA3E0FFC3EF9404EE648067
:10006E00948040030200FCAF1CAE1B12000EEF2466
:10007E0005FFEE3400FE7C007D0A121E598E5C8F49
:10008E005D7B017A00796CC003C002C0017BFF7AF0
:10009E004A792B9000DBEBF0A3EAF0A3E9F0AE5C1B
:1000AE00AF5D7C007D64121E599000DEEEF0A3EF72
:1000BE00F0AE5CAF5D7C007D64121E599000E0ECEA
:1000CE00F0A3EDF0900012E0FF9000E2EFF0900050
:1000DE0011E0FF9000E3EFF0900010E0FF9000E4DD
:1000EE00EFF0D001D002D00312379F020180AF1C77
:1000FE00AE1B12000EEF2432FFEE3400FE7C007DAC
:10010E0064121E598E5C8F5D7B017A00796CC00380
:10011E00C002C0017BFF7A4A794E9000DBEBF0A360
:10012E00EAF0A3E9F0AE5CAF5D7C007D0A121E59C9
:10013E009000DEEEF0A3EFF0AE5CAF5D7C007D0ACA
:10014E00121E599000E0ECF0A3EDF0900012E0FFCB
:10015E009000E2EFF0900011E0FF9000E3EFF090DE
:10016E000010E0FF9000E4EFF0D001D002D00312B7
:10017E00379F751500D3E515648094825042AF15F4
:10018E0090003DE0FE75F003EEA4F58285F083E568
:10019E00822FF582E43583F583E5822429F582E505
:1001AE0083344CF583E493FFAE15EEFD3395E0FCFE
:1001BE00746C2DF58274003CF583EFF0051580B557
:1001CE00C3E51B64809480400302059C90006F740D
:1001DE002DF002059C90003EE0FEA3E0FFEF640AC6
:1001EE004E601190003EE0FEA3E0FFEF640B4E6008
:1001FE00030202877B017A00796CC003C002C00142
:10020E007BFF7A4A79709000DBEBF0A3EAF0A3E96A
:10021E00F090002AE0FEA3E0FF7C007D0A121E593A
:10022E009000DEEEF0A3EFF090002AE0FEA3E0FFD8
:10023E007C007D0A121E599000E0ECF0A3EDF090C8
:10024E00002CE0FEA3E0FF7C007D0A121E599000F8
:10025E00E2EEF0A3EFF090002CE0FEA3E0FF7C00B6
:10026E007D0A121E599000E4ECF0A3EDF0D001D0FF
:10027E0002D00312379F02059C90003EE0FEA3E0E1
:10028E00FFEF640C4E601190003EE0FEA3E0FFEF26
:10029E00640D4E600302032B7B017A00796CC00360
:1002AE00C002C0017BFF7A4A798D9000DBEBF0A390
:1002BE00EAF0A3E9F090002EE0FEA3E0FF7C007DC3
:1002CE000A121E599000DEEEF0A3EFF090002EE021
:1002DE00FEA3E0FF7C007D0A121E599000E0ECF0B8
:1002EE00A3EDF0900030E0FEA3E0FF7C007D0A124B
:1002FE001E599000E2EEF0A3EFF0900030E0FEA366
:10030E00E0FF7C007D0A121E599000E4ECF0A3ED94
:10031E00F0D001D002D00312379F02059C90003E10
:10032E00E0FEA3E0FFEF640E4E601190003EE0FE93
:10033E00A3E0FFEF640F4E60030203F9900034E078
:10034E00FEA3E0FFEF247CF559EE34FCF558AF59CF
:10035E00AE5812000E7C007D0A121E59C006C00750
:10036E00AF59AE5812000E7C007D0A121E59900035
:10037E00E4ECF0A3EDF0D007D0069000E2EEF0A38F
:10038E00EFF07B017A00796CC003C002C0017BFFE5
:10039E007A4A79AA9000DBEBF0A3EAF0A3E9F09099
:1003AE000032E0FEA3E0FF7C007D0A121E59900091
:1003BE00DEEEF0A3EFF0900032E0FEA3E0FF7C0053
:1003CE007D0A121E599000E0ECF0A3EDF0D001D0A2
:1003DE0002D00312379FC3E5586480948040030215
:1003EE00059C900072742DF002059C90003EE0FE7C
:1003FE00A3E0FFEF64104E601190003EE0FEA3E01C
:10040E00FFEF64114E60030204F6900036E0FEA387
:10041E00E0FFEF24F8F55BEE34F8F55A900038E083
:10042E00FEA3E0FFEF247CF559EE34FCF558AF5BEC
:10043E00AE5A12000E7C007D0A121E59C006C0076D
:10044E00AF5BAE5A12000E7C007D0A121E59C0041C
:10045E00C005AF59AE5812000E7C007D0A121E590F
:10046E00C006C007AF59AE5812000E7C007D0A12AE
:10047E001E599000E4ECF0A3EDF0D007D0069000EA
:10048E00E2EEF0A3EFF0D005D0049000E0ECF0A384
:10049E00EDF0D007D0069000DEEEF0A3EFF07B017A
:1004AE007A00796CC003C002C0017BFF7A4A79C71B
:1004BE009000DBEBF0A3EAF0A3E9F0D001D002D07C
:1004CE000312379FC3E55A648094805006900071E2
:1004DE007445F0C3E55864809480400302059C90F7
:1004EE0000777453F002059C7B017A00796CC0038F
:1004FE00C002C0017BFF7A4A79E49000DBEBF0A3E7
:10050E00EAF0A3E9F0900013E0FF9000DEEFF09028
:10051E000015E0FF9000DFEFF0900012E0FF90007A
:10052E00E0EFF0900011E0FF9000E1EFF09000108E
:10053E00E0FF9000E2EFF0D001D002D00312379F1F
:10054E00751500D3E515648094825042AF15900066
:10055E0014E0FE75F003EEA4F58285F083E5822F9C
:10056E00F582E43583F583E58224BEF582E5833496
:10057E004BF583E493FFAE15EEFD3395E0FC746E00
:10058E002DF58274003CF583EFF0051580B59000D3
:10059E0028E0FEA3E0FFC3EF9402EE648094805047
:1005AE003290003EE0FEA3E0FFC3EF940AEE6480BB
:1005BE009480401390003EE0FEA3E0FFD3EF941131
:1005CE00EE64809480400C90007E7444F090007F26
:1005DE007445F07F00125BC6751500D3E515648077
:1005EE009493501AAF15EF3395E0FE746C2FF5828D
:1005FE0074003EF583E0FF125B8D051580DD200E45
:10060E000302080CC20E90003EE0FEA3E0FFC3EF13
:10061E00940AEE64809480401590003EE0FEA3E0C4
:10062E00FFD3EF9411EE648094805002C2129001B9
:10063E00CAE0F8A3E0F9A3E0FAA3E0FB900004E01F
:10064E00FCA3E0FDA3E0FEA3E0FF1219F4126A5230
:10065E007B007A00792078411218EB7B007A0079C2
:10066E0000783F1217FA121B4D8E588F599001CAFF
:10067E00E0F8A3E0F9A3E0FAA3E0FB900068E0FC49
:10068E00A3E0FDA3E0FEA3E0FF1219F4126A527B71
:10069E00007A007900783F1217FA121B4D8E628F86
:1006AE00637B017A007984C003C002C0017BFF7AAC
:1006BE004B79099000DBEBF0A3EAF0A3E9F090018F
:1006CE00CAE0F8A3E0F9A3E0FAA3E0FB90000CE087
:1006DE00FCA3E0FDA3E0FEA3E0FF1219F49000DE00
:1006EE00121FA5AE58AF597C007D0A121E599000FC
:1006FE00E2EEF0A3EFF0AE58AF597C007D0A121E69
:10070E00599000E4ECF0A3EDF09000E6E562F0A362
:10071E00E563F0D001D002D00312379F7F007E0038
:10072E007D007C00900004E0F8A3E0F9A3E0FAA3BA
:10073E00E0FB121A91500690008A742DF075150088
:10074E00D3E515648094855042AF15900029E0FEE4
:10075E0075F006EEA4F58285F083E5822FF582E42E
:10076E003583F583E58224E6F582E583344BF58304
:10077E00E493FFAE15EEFD3395E0FC74902DF582FB
:10078E0074003CF583EFF0051580B5900028E0FE6F
:10079E00A3E0FFC3EF9402EE64809480400E9000BD
:1007AE00967420F09000977420F080217F007E00D8
:1007BE007D007C00900068E0F8A3E0F9A3E0FAA3C6
:1007CE00E0FB121A915006900095742DF0E56A64C4
:1007DE0001602B7F40125BC6751500D3E515648052
:1007EE009493501AAF15EF3395E0FE74842FF58273
:1007FE0074003EF583E0FF125B8D051580DD200F42
:10080E0003020917C20F900022E0FEA3E0FFEF24BF
:10081E009CFFEE34FFFE12000E8E5A8F5B9000246A
:10082E00E0FEA3E0FFEF249CFFEE34FFFE12000E6D
:10083E008E588F597B017A00799CC003C002C0018B
:10084E007BFF7A4B79279000DBEBF0A3EAF0A3E96C
:10085E00F0AE5AAF5B7C007D0A121E599000DEEEA0
:10086E00F0A3EFF0AE5AAF5B7C007D0A121E5990DA
:10087E0000E0ECF0A3EDF0AE58AF597C007D0A120B
:10088E001E599000E2EEF0A3EFF0AE58AF597C0087
:10089E007D0A121E599000E4ECF0A3EDF0D001D0C9
:1008AE0002D00312379F900022E0FEA3E0FFC3EFB9
:1008BE009464EE64809480500690009D742DF090A8
:1008CE000024E0FEA3E0FFC3EF9464EE6480948006
:1008DE0050069000A3742DF0E56A6401602B7F141E
:1008EE00125BC6751500D3E51564809493501AAF4C
:1008FE0015EF3395E0FE749C2FF58274003EF58360
:10090E00E0FF125B8D051580DD201003020B60C227
:10091E001020B338E5462464FFE5453400FE900010
:10092E0022E0FCA3E0FDC3EF9DF561EE9CF560E5D2
:10093E00412464FFE5403400FE900024E0FCA3E077
:10094E00FDC3EF9DF55FEE9CF55E800C85456085E1
:10095E00466185405E85415F900027E0FFEF904C39
:10096E00F193FFEF3395E0FEAC4EAD4F121E478E66
:10097E00438F44AF5FAE5E12000E7C007D0A121EE6
:10098E0059C006C007AF5FAE5E12000E7C007D0A36
:10099E00121E599000E4ECF0A3EDF0D007D00690B3
:1009AE0000E2EEF0A3EFF07B017A0079B4C003C051
:1009BE0002C0017BFF7A4B79499000DBEBF0A3EA92
:1009CE00F0A3E9F0AE60AF617C007D0A121E599073
:1009DE0000DEEEF0A3EFF0AE60AF617C007D0A1298
:1009EE001E599000E0ECF0A3EDF0AE43AF447C0056
:1009FE007D0A121E599000E6EEF0A3EFF0AE43AF63
:100A0E00447C007D0A121E599000E8ECF0A3EDF034
:100A1E00D001D002D00312379FC3E540648094808A
:100A2E0050069000BA742DF0A218B39218E508542F
:100A3E000CFFEFB408082018059000C4E4F0E50898
:100A4E00540CFFEFB404092018069000C47401F092
:100A5E00E508540CFFEFB40C093017069000C4746F
:100A6E002AF0E5085403FFEFB4020930180690008F
:100A7E00C37402F0E5085403FFEFB4010930180601
:100A8E009000C37403F0E5085403FFEFB40309307C
:100A9E0017069000C3742AF090003EE0FEA3E0FF1C
:100AAE00EF64124E6003020B35751500D3E5156425
:100ABE008094935042AF1590003BE0FE75F014EE1B
:100ACE00A4F58285F083E5822FF582E43583F583E4
:100ADE00E582243CF582E583344CF583E493FFAE46
:100AEE0015EEFD3395E0FC74B42DF58274003CF5E3
:100AFE0083EFF0051580B5AE43AF447C007D0A123E
:100B0E001E59EF2430FF9000C5EFF09000C6742EF2
:100B1E00F0AE43AF447C007D0A121E59AF05EF24A0
:100B2E0030FF9000C7EFF07F54125BC6751500D3EF
:100B3E00E51564809493501AAF15EF3395E0FE746B
:100B4E00B42FF58274003EF583E0FF125B8D051520
:100B5E0080DDE56AB4011490003FE0FFEF904CDDBC
:100B6E0093FF125BC6125BAB125BBD301103020C1E
:100B7E00C37B017A00796CC003C002C0017BFF7A8F
:100B8E004B796A9000DBEBF0A3EAF0A3E9F0D00119
:100B9E00D002D00312379F7B017A007984C003C044
:100BAE0002C0017BFF7A4B797F9000DBEBF0A3EA6A
:100BBE00F0A3E9F0D001D002D00312379F7B017A67
:100BCE0000799CC003C002C0017BFF7A4B799490E0
:100BDE0000DBEBF0A3EAF0A3E9F0D001D002D003E2
:100BEE0012379F7B017A0079B4C003C002C0017B2B
:100BFE00FF7A4B79A99000DBEBF0A3EAF0A3E9F0C2
:100C0E00D001D002D00312379F7F00125BC675153C
:100C1E0000D3E51564809493501AAF15EF3395E029
:100C2E00FE746C2FF58274003EF583E0FF125B8D2F
:100C3E00051580DD7F40125BC6751500D3E5156482
:100C4E00809493501AAF15EF3395E0FE74842FF510
:100C5E008274003EF583E0FF125B8D051580DD7F0B
:100C6E0014125BC6751500D3E51564809493501A63
:100C7E00AF15EF3395E0FE749C2FF58274003EF5B0
:100C8E0083E0FF125B8D051580DD7F54125BC67508
:100C9E001500D3E51564809493501AAF15EF339574
:100CAE00E0FE74B42FF58274003EF583E0FF125B14
:060CBE008D051580DD220A
:10695A00014900014700014800014200C117C11660
:02696A00C11555
:106A1F00752400D3E524648094A75004052480F3E3
:016A2F002244
:106A3000752500D3E525648094935004052580F3E3
:016A40002233
:106A4100752600D3E5266480949E5004052680F3C4
:016A51002222
:105D0A00C290126A1F752C1F752B00E52BD39407BE
:105D1A005011E52CC313F52CA2D79290126A1F05D5
:105D2A002B80E8D290126A1FD2927527037528E851
:105D3A00752C00309110E52815287002152714FFDC
:105D4A00AE27EF4E70ED126A30752B00E52BD39417
:105D5A00075013126A1FE52CC313F52C3091034325
:105D6A002C80052B80E6126A1FAF2C7E00EF752A65
:105D7A0000F5297527037528E8752C00309110E580
:105D8A002815287002152714FFAE27EF4E70ED1262
:105D9A006A30752B00E52BD394075013126A1FE55E
:105DAA002CC313F52C309103432C80052B80E6126B
:105DBA006A1FAF2C7E00EF252AF52AEE3529F52930
:105DCA00C3E529648094805006752900752A00D39A
:105DDA00E52A940FE5296480948E400675290E758C
:105DEA002A0FC29220B20DC3740F952AF52A740E97
:085DFA009529F529AE29AF2A15
:015E0200227D
:105EF300C294126A1F75321F753100E531D39407BE
:105F03005011E532C313F532A2D79294126A1F05DA
:105F13003180E8D294126A1FD296752D03752EE84C
:105F2300753200309510E52E152E7002152D14FFD5
:105F3300AE2DEF4E70ED126A30753100E531D3941A
:105F4300075013126A1FE532C313F532309503432A
:105F53003280053180E6126A1FAF327E00EF753062
:105F630000F52F752D03752EE8753200309510E579
:105F73002E152E7002152D14FFAE2DEF4E70ED125F
:105F83006A30753100E531D394075013126A1FE567
:105F930032C313F532309503433280053180E61264
:105FA3006A1FAF327E00EF2530F530EE352FF52F27
:105FB300C3E52F648094805006752F00753000D39D
:105FC300E530940FE52F6480948E4006752F0E758F
:085FD300300FC296AE2FAF3073
:015FDB0022A3
:1069B800125D0A8E458F46125EF3C374089FFF74FA
:1069C800079EFE12000EC374849FF54174039EF562
:0869D80040754E00754F0122CD
:10609900D290D294D291D29575540075550075500D
:1060A90000755100753300D3E533648094895049F4
:1060B900126A41C290C294126A41C3E53364809462
:1060C900895004D290D294E5552555F555E55435B6
:1060D90054F554E5512551F551E5503550F5502009
:1060E90091080555E555700205542095080551E5B7
:1060F9005170020550053380AEC290C294754E00AE
:10610900754F05AE54AF557C007D05121E478E456F
:106119008F4620B20DC3740B9546F546740E95450E
:10612900F545C374689551FF74019550FE12000E30
:10613900C374B49FF551E49EF550AE50AF517C0045
:096149007D05121E478E408F41B6
:01615200222A
:10615300D290D294D291D295755400755500755052
:1061630000755100753400D3E5346480948A504936
:10617300126A41C290C294126A41C3E534648094A6
:106183008A5004D290D294E5552555F555E55435FA
:1061930054F554E5512551F551E5503550F550204E
:1061A30091080555E555700205542095080551E5FC
:1061B3005170020550053480AEC290C294754E00F2
:1061C300754F02E55525E0F546E55433F54520B214
:1061D3000DC3740E9546F546740E9545F545C37487
:1061E300849551FF74039550FE12000EC374C29F31
:1061F300F55174019EF550E55125E0F541E5503325
:02620300F54064
:016205002276
:10656800D290D294D291D295755400755500755039
:1065780000755100753500D3E5356480948B50491A
:10658800126A41C290C294126A41C3E5356480948C
:106598008B5004D290D294E5552555F555E55435E0
:1065A80054F554E5512551F551E5503550F5502035
:1065B80091080555E555700205542095080551E5E3
:1065C8005170020550053580AEC290C294754E00D8
:1065D800754F0185544585554620B20DC3740F95F6
:1065E80046F546740E9545F545C374089551FF74F4
:1065F800079550FE12000EC374849FF54174039EE4
:02660800F5405B
:01660A00226D
:10562500D292D291755400755500126A419001EDE0
:10563500E4F09001EDE0FFD3EF6480948F5029D220
:1056450090126A41C290126A41E5552555F555E516
:10565500543554F5542091080555E5557002055407
:105665009001EDE004F080CAC290C292E555AE54B7
:105675007806CEC313CE13D8F9F5558E54AC54AD78
:1056850055E4121B147B007A00793478441218EB28
:105695007B007A00798078441219F4121B4D7C0046
:1056A5007D05121E478E458F4620B20DC3740B959E
:1056B50046F546740E9545F545126A41754E0075D9
:1056C5004F05D296D295755000755100126A4190DA
:1056D50001EDE4F09001EDE0FFD3EF6480948F508D
:1056E50029D294126A41C294126A41E5512551F5B5
:1056F50051E5503550F5502095080551E55170029A
:1057050005509001EDE004F080CAC294C296E551BF
:10571500AE507806CEC313CE13D8F9F5518E50C3CB
:10572500E49551FF74029550FE12000EC3E49FFDEF
:1057350074019EFCEC121B147B007A0079347844CA
:105745001218EB7B007A00798078441219F4121B49
:0C5755004D7C007D05121E478E408F41E8
:015761002225
:10576200D292D291755400755500126A419001EEA1
:10577200E4F09001EEE0FFD3EF6480948F5029D2E1
:1057820090126A41C290126A41E5552555F555E5D8
:10579200543554F5542091080555E55570020554C9
:1057A2009001EEE004F080CAC290C292E555AE5478
:1057B2007805CEC313CE13D8F9F5558E54AC54AD3B
:1057C20055E4121B147B007A0079E178441218EB3D
:1057D2007B007A00790078451219F4121B4DEF25EF
:1057E200E0F546EE33F54520B20DC3740E9546F54D
:1057F20046740E9545F545126A41754E00754F0285
:10580200D296D295755000755100126A419001EE00
:10581200E4F09001EEE0FFD3EF6480948F5029D240
:1058220094126A41C294126A41E5512551F551E53B
:10583200503550F5502095080551E551700205503C
:105842009001EEE004F080CAC294C296E551AE50D7
:105852007805CEC313CE13D8F9F5518E50C3E49513
:1058620051FF74049550FE12000EC3E49FFD7402B2
:105872009EFCEC121B147B007A0079E1784412182A
:10588200EB7B007A00790078451219F4121B4DEF78
:0858920025E0F541EE33F5407D
:01589A0022EB
:10589B00D292D291755400755500126A419001EF66
:1058AB00E4F09001EFE0FFD3EF6480948F5029D2A6
:1058BB0090126A41C290126A41E5552555F555E59E
:1058CB00543554F5542091080555E555700205548F
:1058DB009001EFE004F080CAC290C292E554C4F884
:1058EB0054F0C868F554E555C4540F48F555AC54FD
:1058FB00AD55E4121B147B007A00796178451218C0
:10590B00EB7B007A00798078451219F4121B4D8ECF
:10591B00458F4620B20DC3740F9546F546740E9510
:10592B0045F545126A41754E00754F01D296D295D9
:10593B00755000755100126A419001EFE4F090012F
:10594B00EFE0FFD3EF6480948F5029D294126A4119
:10595B00C294126A41E5512551F551E5503550F588
:10596B00502095080551E551700205509001EFE06C
:10597B0004F080CAC294C296E550C4F854F0C868CB
:10598B00F550E551C4540F48F551C3E49551FF74DC
:10599B00089550FE12000EC3E49FFD74049EFCECB0
:1059AB00121B147B007A00796178451218EB7B008F
:1059BB007A00798078451219F4121B4D8E408F4175
:0159CB0022B9
:105C0B00D290D294D291D29575540075550075509F
:105C1B0000755100753600D3E5366480948B505374
:105C2B00C290C294753700D3E537648094825004D8
:105C3B00053780F3C3E5366480948B5004D290D241
:105C4B0094E5552555F555E5543554F554E5512551
:105C5B0051F551E5503550F5502091080555E55556
:105C6B00700205542095080551E551700205500549
:105C7B003680A4C290C294754E00754F01AF55AEDD
:105C8B0054126A078E548F55AF51AE50126A078E5D
:105C9B00508F51AC54AD55E4121B147B007A007934
:105CAB006178451218EB7B007A00798078451219E0
:105CBB00F4121B4D8E458F4620B20DC3740F9546C3
:105CCB00F546740E9545F545C3E49551FF7408955B
:105CDB0050FE12000EC3E49FFD74049EFCEC121BDD
:105CEB00147B007A00796178451218EB7B007A00FF
:0E5CFB00798078451219F4121B4D8E408F41AE
:015D09002277
:1043D00075080FE55724F8F54BE55634F8F54AE52E
:1043E0004624F8F54DE54534F8F54CC3E54A6480BC
:1043F0009480500C7410254BF54B740E354AF54AD9
:10440000C3E54C64809480500C7410254DF54D74B8
:104410000E354CF54C900038E0FEA3E0FFC3EF945E
:1044200084EE648094834025900022E0FEA3E0FFA8
:10443000E5572FFFE5563EFEEF249CFFEE34FFFECE
:10444000C3EF9546F539EE9545F538802390002267
:10445000E0FEA3E0FFE54B2FFFE54A3EFEEF249C84
:10446000FFEE34FFFEC3EF954DF539EE954CF53870
:10447000D3E5539400E55264809480402590002455
:10448000E0FEA3E0FFE5532FFFE5523EFEEF249C44
:10449000FFEE34FFFEC3EF9541F53BEE9540F53A54
:1044A000801B900024E0FEA3E0FFEF249CFFEE348D
:1044B000FFFEC3EF9541F53BEE9540F53A2017031B
:1044C000024702AE43AF447C007D02121E59D3E581
:1044D000399FEE6480F8E53864809840289001F0B8
:1044E000E0FFEF20E5067549007548000549AF4932
:1044F000EFD394504003754950E549C3940A4054A2
:1045000053080E804FAE43AF447C007D02121E590B
:10451000C3E49FFFE49EFEC3E5399FEE6480F8E5A7
:104520003864809850289001F0E0FFEF20E4067591
:1045300049007548000549AF49EFD39450400375D1
:104540004950E549C3940A400B53080D800675494C
:1045500000754800AE43AF447C007D02121E59D363
:10456000E53B9FEE6480F8E53A648098402890012E
:10457000F0E0FFEF20E7067547007542000547AF02
:1045800047EFD394504003754750E547C3940A4022
:104590006153080B805CAE43AF447C007D02121E69
:1045A00059C3E49FFFE49EFEC3E53B9FEE6480F8A1
:1045B000E53A6480985035D3E5419400E540648045
:1045C000948040289001F0E0FFEF20E60675470058
:1045D0007542000547AF47EFD394504003754750ED
:1045E000E547C3940A400B530807800675470075DA
:1045F0004200AF39AE3812000E8E3C8F3DC3742896
:10460000953DFFE4953CFEEF7802C333CE33CED820
:10461000F9FFAD487C00C3EF9DF53FEE9CF53EC32E
:10462000E53E648094805006753E00753F00E54984
:10463000C39450501DAF497E007C007D7F121E4701
:104640007C007D50121E59EF2480FFEF64FFF5FAC5
:104650008027C3E53D9428E53C648094805017E5AD
:1046600048C394A050100548C3E53E648094804040
:1046700008853FFA800375FA00AF3BAE3A12000E90
:104680008E3C8F3DC37428953DFFE4953CFEEF784A
:1046900002C333CE33CED8F9FFAD427C00C3EF9DC9
:1046A000F53FEE9CF53EC3E53E6480948050067570
:1046B0003E00753F00E547C39450501DAF477E0054
:1046C0007C007D7F121E477C007D50121E59EF2416
:1046D00080FFEF64FFF5FE803BC3E53D9428E53C99
:1046E000648094805017E542C394A050100542C3E3
:1046F000E53E64809480401C853FFE801775FE0077
:10470000801275490075480075470075420075FABA
:104710000075FE00E508C454F0FFEF240FFF900180
:0A472000F0EFF09001F0E0FF8FA031
:01472A00226C
:106980004310000043D8000044A20000451100005D
:1069900045B400004622000000C700C70002000AFC
:1069A0000E0F03840E0F038400010001000000009D
:0869B0000000000000000000DF
:10696C00011400011663011200011700011A00C185
:03697C000CC18BC0
:03000300025FDCBD
:105FDC00C0E0C083C08263A201C083C082C0D07500
:105FEC00D000C006C007200B4F200C4CD2B330B3EE
:105FFC00020512051AAF1AC3EF64809488401CAFD7
:10600C0017EF3395E0FE74402FF58274003EF58354
:10601C00E512F07512000517751A00E5122512F538
:10602C0012C3E51764809484404F751700D20C900E
:10603C000048E0FF8F128041200B3E300C3BE512F4
:10604C002512F512A2D792B3051AAF1AC3EF6480CA
:10605C009488401A0517AF17EF3395E0FE74482F5C
:10606C00F58274003EF583E0FF8F12751A00C3E5CC
:10607C0017648094A04002D20BD007D006D0D0D0A9
:0D608C0082D08363A201D082D083D0E032A5
:104F2300900048E556F0A3E557F0E5532484FFE5E8
:104F3300523403FE90004AEEF0A3EFF090004CE5EC
:104F430045F0A3E546F0E5412484FFE5403403FE44
:104F530090004EEEF0A3EFF0E50B2484FFE50A3456
:104F630003FE900050EEF0A3EFF0900022E0FEA3CA
:104F7300E0FF900052EEF0A3EFF0900024E0FEA3D8
:104F8300E0FF900054EEF0A3EFF0900028E0FEA3C2
:104F9300E0FF900056EEF0A3EFF0900058E543F0E9
:104FA300A3E544F030170B90005AE4F0A37401F02A
:104FB300800890005AE4F0A3E4F0900015E0FFEFBE
:104FC3003395E0FE90005CEEF0A3EFF0900014E068
:104FD300FFEF3395E0FE90005EEEF0A3EFF090005C
:104FE30013E0FFEF3395E0FE900060EEF0A3EFF0E7
:104FF300900012E0FFEF3395E0FE900062EEF0A325
:10500300EFF0900011E0FFEF3395E0FE900064EEC7
:10501300F0A3EFF0900041E0F516900040E4F0A318
:105023007463F0C3E516648094884003025108C397
:10503300E516648094805003025108900042E0F525
:1050430018A3E0F519AF16EF3395E0FEEF25E0FF67
:10505300EE33FE74982FF58274693EF583E493FE74
:10506300740193FFD3E5199FEE6480F8E51864801B
:10507300984021AF16EF3395E0FEEF25E0FFEE33C6
:10508300FE74982FF58274693EF583E493F51874E2
:105093000193F519AF16EF3395E0FEEF25E0FFEE30
:1050A30033FE74A82FF58274693EF583E493FE748E
:1050B3000193FFC3E5199FEE6480F8E518648098B7
:1050C3005021AF16EF3395E0FEEF25E0FFEE33FE00
:1050D30074A82FF58274693EF583E493F51874017F
:1050E30093F519AF16EF3395E0FEEF25E0FFEE33AE
:1050F300FE74222FF58274003EF583E518F0A3E5D4
:1051030019F0124DF8E516B40805A217B392172249
:03002B0002620668
:10620600C0E0C0F0C083C08263A201C083C082C068
:10621600D075D000C000C001C002C003C004C005D4
:10622600C006C007C2CF75A61E75A6E11509AF093F
:10623600EF705E75090490003AE0FEA3E0FFEF8E72
:10624600F0122028626E000062730001627800027C
:10625600627D00036282000462870005628C00068C
:1062660062910007000062941260998021126153C6
:10627600801C1265688017125C0B80121269B88048
:106286000D1256258008125762800312589B12433E
:10629600D0D007D006D005D004D003D002D001D08C
:1062A60000D0D0D082D08363A201D082D083D0F038
:0362B600D0E03203
:0300230002685020
:10685000C0E0C0F0C083C08263A201C083C082C018
:10686000D075D000C000C001C002C003C004C00584
:10687000C006C007C2AC30981AC298E599B43F036D
:10688000125113E599B4210B1252F9D20DD20ED246
:106890000FD210C299D2ACD007D006D005D004D008
:1068A00003D002D001D000D0D0D082D08363A20127
:0968B000D082D083D0F0D0E03298
:03000B000262B9D5
:1062B900C0E0C0F0C083C08263A201C083C082C0B5
:1062C900D075D000C000C001C002C003C004C00521
:1062D900C006C007758A00758C4C75A61E75A6E1A7
:1062E9000514AF14C3EF6480948A4016300B1375FC
:1062F9001400751700751A00C20CC20B7512001232
:106309004F23E51375F007121DCDAFF0EF701E1284
:106319003BBD301104D20DD210E56A60073011047B
:10632900D20ED20F12002E124D49124E051513AF7F
:1063390013EF700C75134ED211301104D20ED20F17
:10634900D007D006D005D004D003D002D001D000A8
:10635900D0D0D082D08363A201D082D083D0F0D0B4
:02636900E03220
:1021C200758FFF758921758DFF438780759850D271
:1021D2008CD28ED2CA75CB4C75CA0043B81143B7A4
:1021E20021D28875D90243D84075DA4275DE42C2DF
:1021F200117513467509017F02125B55125BA275B8
:102202006B00900040E4F0A37463F020A003126717
:10221200D675A8B275A707E56A70FC900036E0FC97
:10222200A3E0FDEC121B147B007A007920784112A6
:1022320019F47B007A00793478C31217FA9001CA34
:10224200E0F8A3E0F9A3E0FAA3E0FB1218EB900098
:102252001E121FA5900038E0FCA3E0FDEC121B1437
:102262007B007A00792078411219F47B007A007998
:10227200B478C21217FA9001CAE0F8A3E0F9A3E019
:10228200FAA3E0FB1218EB90001A121FA59000119E
:10229200E0FCEC121B197B007A0079B47844121925
:1022A200F4C004C005C006C007900012E0FCEC12A6
:1022B2001B197B007A0079C078411219F4A804A98D
:1022C20005AA06AB07D007D006D005D0041217FA2C
:1022D200C004C005C006C007900010E0FCEC121B51
:1022E200197B007AC079A878471219F4A804A905C5
:1022F200AA06AB07D007D006D005D0041217FA9071
:102302000044121FA5900014E0FFEF3395E0FEFD9C
:10231200FCEF2409FFEE3400FEED3400FDEC340046
:10232200FC7B0C7A00790078001268B9A804A90530
:10233200AA06AB07900015E0FFEF3395E0FEFDFC27
:10234200EF24D0FFEE3407FEED3400FDEC3400FC48
:10235200EB2FFFEA3EFEE93DFDE83CFC7B077A00FD
:1023620079007800121EA57B047A007900780012A9
:1023720068B9C004C005C006C007900015E0FFEFB1
:102382003395E0FEFDFC7B6F7A0179007800121E26
:10239200A5D003D002D001D000C3EF9BFFEE9AFE7E
:1023A200ED99FDEC98FCC004C005C006C007900082
:1023B20014E0FFEF3395E0FEFDFC7B137A01790018
:1023C2007800121EA57B097A00790078001268B99C
:1023D200A804A905AA06AB07D007D006D005D004E9
:1023E200EB2FFBEA3EFAE93DF9E83CF8900013E0F6
:1023F200FFEF3395E0FEFDFCEB2FFFEA3EFEE93DE9
:10240200FDE83CFCEF247AF511EE34E0F510ED34F2
:1024120000F50FEC3400F50E900028E0FEA3E0FF7B
:10242200EF64014E70487B017A007908C003C00254
:10243200C0017B017A007968900193EBF0A3EAF086
:10244200A3E9F0AF11AE10AD0FAC0E900196121FC2
:10245200A5900044E0FCA3E0FDA3E0FEA3E0FF9012
:10246200019A121FA5D001D002D003124008900099
:1024720028E0FEA3E0FFEF4E60030226477B017ACD
:10248200007908C003C002C0017B017A007968901C
:10249200010BEBF0A3EAF0A3E9F0AF11AE10AD0F20
:1024A200AC0E90010E121FA5900044E0FCA3E0FDCB
:1024B200A3E0FEA3E0FF900112121FA5D001D002FB
:1024C200D003122A1C90001AE0FCA3E0FDA3E0FE58
:1024D200A3E0FF1254E57B547AE379457840121861
:1024E200EBC004C005C006C007900016E0FCA3E0E4
:1024F200FDA3E0FEA3E0FF1254FBA804A905AA066F
:10250200AB07D007D006D005D0041218EBC004C028
:1025120005C006C007900068E0FCA3E0FDA3E0FE52
:10252200A3E0FF1254E5A804A905AA06AB07D00749
:10253200D006D005D0041218EBC004C005C006C0F6
:1025420007AF11AE10AD0FAC0EC004C005C006C07F
:10255200077FAB7EAA7D2A7C3C900044E0F8A3E092
:10256200F9A3E0FAA3E0FB1217FA900146121FA5A5
:10257200D007D006D005D004120CC4C004C005C0D8
:1025820006C007AF11AE10AD0FAC0EC004C005C03F
:1025920006C0077FAB7EAA7D2A7CBC900044E0F88F
:1025A200A3E0F9A3E0FAA3E0FB1217FA90014612A6
:1025B2001FA5D007D006D005D004120CC4D003D07A
:1025C20002D001D0001217F67B007A007987784397
:1025D2001219F4A804A905AA06AB07D007D006D0A1
:1025E20005D0041217FA7B007A00797A784412181F
:1025F200EB121B4D8E0C8F0DAC0CAD0DEC121B149F
:10260200C004C005C006C00790003CE0FEA3E0FF86
:10261200EF7802C333CE33CED8F9FF74802FF58220
:1026220074693EF583121F75D007D006D005D00419
:102632001218EB7B007A00797A78441219F4121B93
:102642004D8E1B8F1C900028E0FEA3E0FFEF64027A
:102652004E7014900068121FB13F82D0E5900008BE
:10266200121FB140C39DB2900028E0FEA3E0FFEF2D
:1026720064034E7014900068121FB13F3566CF900C
:102682000008121FB140A73B64900028E0FEA3E0BF
:10269200FFEF64044E7014900068121FB1BF018FE7
:1026A200C5900008121FB140953F7D900028E0FEC2
:1026B200A3E0FFEF64054E7014900068121FB13E54
:1026C200C44D01900008121FB13FB916879000282F
:1026D200E0FEA3E0FFEF64064E7014900068121F44
:1026E200B13F32B6AE900008121FB1401F2B0290CC
:1026F2000028E0FEA3E0FFEF64074E70149000682C
:10270200121FB100000000900008121FB140BC7AF5
:10271200E1900028E0FEA3E0FFEF64084E706790AE
:102722000032E0FCA3E0FDEC121B147B007A00797E
:102732002078411219F49001CAE0F8A3E0F9A3E06D
:10274200FAA3E0FB1218EB900008121FA5900034C8
:10275200E0FCA3E0FDEC121B147B007A00792078E8
:10276200411219F47B007A0079B478C21217FA90F8
:1027720001CAE0F8A3E0F9A3E0FAA3E0FB1218EB28
:10278200900068121FA5900028E0FEA3E0FFC3EFAF
:102792009409EE64809480400302289B900044E0F8
:1027A200FCA3E0FDA3E0FEA3E0FFC004C005C00659
:1027B200C007AF11AE10AD0FAC0E9001B6121FA53F
:1027C200D007D006D005D00412472B900170121FFB
:1027D200A57B017A00790CC003C002C0017B017A9B
:1027E20000790090016DEBF0A3EAF0A3E9F090000C
:1027F20008E0FCA3E0FDA3E0FEA3E0FF9001741259
:102802001FA5900068E0FCA3E0FDA3E0FEA3E0FFAB
:10281200900178121FA5D001D002D003123223906A
:102822000028E0FEA3E0FFEF4E705A900000E0FCAB
:10283200A3E0FDA3E0FEA3E0FF1254E57B007A5083
:1028420079C778451218EBC004C005C006C00790CE
:1028520000D0121FB148B98C00D007D006D005D0E5
:10286200041266A8A804A905AA06AB07900000E016
:10287200FCA3E0FDA3E0FEA3E0FF1217F690000424
:10288200121FA58014900000E0FCA3E0FDA3E0FE6F
:10289200A3E0FF900004121FA5900028E0FEA3E031
:1028A200FFEF64094E705C90002EE0FCA3E0FDECAB
:1028B200121B147B007A00792078411219F49001DE
:1028C200CAE0F8A3E0F9A3E0FAA3E0FB1218EB9048
:1028D200000C121FA5900030E0FCA3E0FDEC121BDF
:1028E200147B007A00792078411219F49001CAE031
:1028F200F8A3E0F9A3E0FAA3E0FB1218EB900004BE
:10290200121FA5900028E0FEA3E0FFEF640A4E70BC
:102912005C90002AE0FCA3E0FDEC121B147B007A21
:1029220000792078411219F49001CAE0F8A3E0F985
:10293200A3E0FAA3E0FB1218EB90000C121FA59083
:10294200002CE0FCA3E0FDEC121B147B007A007962
:102952002078411219F49001CAE0F8A3E0F9A3E04B
:10296200FAA3E0FB1218EB900004121FA59001CA13
:10297200E0F8A3E0F9A3E0FAA3E0FB90000CE0FC8E
:10298200A3E0FDA3E0FEA3E0FF1219F47BCD7ACC15
:10299200794C783D1217FA7B007A0079207841123F
:1029A20018EB121B4D8E568F579001CAE0F8A3E028
:1029B200F9A3E0FAA3E0FB900004E0FCA3E0FDA38E
:1029C200E0FEA3E0FF1219F47BCD7ACC794C783D7E
:1029D2001217FA7B007A00792078411218EB121B49
:1029E2004D8E528F537F007E007D207C4190006887
:1029F200E0F8A3E0F9A3E0FAA3E0FB1218EB9001E0
:102A0200CAE0F8A3E0F9A3E0FAA3E0FB1219F4127A
:0A2A12001B4D8E0A8F0B02221922C1
:105AEE00EFC0E0C283740F125B237430125B2D740F
:105AFE0005125B237430125B2D7401125B2374301C
:105B0E00125B2D7401125B23D0E014600274084402
:105B1E0020125B3B227D000000DDFCD5E0F7225415
:105B2E00F053800F4280C282D283C28322C282800F
:105B3E0002D282C0E0125B49D0E0C454F053800F11
:105B4E004280D283C28322125AEE125B87740612EF
:105B5E005B3B125B87740E125B3B125B8774011208
:105B6E005B3B125B877440125B3B125BD4125B870C
:105B7E007480125B3B125BB422740A125B2322EF19
:105B8E00C0E0125B87D0E0125B3F22125B8774028B
:105B9E00125B3B22125B877401125B3B22125B8706
:105BAE00740E125B3B22125B87740C125B3B22124B
:105BBE005B87740F125B3B22EFC0E0125B87D0E075
:105BCE004480125B3B22905BE37E28E493FF125BE2
:105BDE008DA3DEF7220004040E0E1F1F00001F1FF0
:105BEE000E0E04040000101C1F1C10000000010704
:0D5BFE001F070100000E11171917110E00EE
:106A07007A107B00EE6BFB8BF053F080ABF033EF2B
:086A170033FFEE33FEDAEE223C
:106745009001EBEEF0A3EFF09001EBE0FEA3E0FF8C
:106755007C037DE8121E59EF2430F5993099FDC26E
:10676500999001EBE0FEA3E0FF7C037DE8121E5942
:106775007E007F64CFCDCFCECCCE121E59EF243014
:10678500F5993099FDC2999001EBE0FEA3E0FF7CFD
:10679500007D64121E597E007F0ACFCDCFCECCCEB0
:1067A500121E59EF2430F5993099FDC2999001EBED
:1067B500E0FEA3E0FF7C007D0A121E59AF05EF2421
:1067C50030F5993099FDC2997599003099FDC299B6
:0167D50022A1
:105113009001E1121FB1000186A020983E9001E1A9
:10512300E0FCA3E0FDA3E0FEA3E0FFEC4D4E4F60E7
:105133002A9001E1E0FCA3E0FDA3E0FEA3E0FF7BF6
:10514300FF7AFF79FF78FFEF2BFFEE3AFEED39FD93
:10515300EC38FC9001E1121FA580BFC298AF99EF14
:1051630012200251B86151C46251D06351D86451C5
:10517300E46551F06651FC67520868521469522085
:105183006A522C6B52386C52446D52506E525E6FA1
:10519300526670527471527C72528A735292745274
:1051A300A57552B37652C17752CF7852DD7952EB5F
:1051B3007A000052F8900022E0FEA3E0FF12674558
:1051C30022900024E0FEA3E0FF12674522AF44AE25
:1051D3004312674522900028E0FEA3E0FF126745D3
:1051E3002290002AE0FEA3E0FF1267452290002CE4
:1051F300E0FEA3E0FF1267452290002EE0FEA3E04D
:10520300FF12674522900030E0FEA3E0FF126745DE
:1052130022900032E0FEA3E0FF12674522900034A3
:10522300E0FEA3E0FF12674522900036E0FEA3E014
:10523300FF12674522900038E0FEA3E0FF126745A6
:105243002290003AE0FEA3E0FF12674522E50D2419
:1052530088FFE50C3413FE12674522AF46AE4512B4
:10526300674522E5412484FFE5403403FE12674588
:1052730022AF57AE5612674522E5532484FFE55209
:105283003403FE12674522AF0BAE0A126745223084
:1052930017087F017E00126745227F007E00126798
:1052A3004522900010E0FFEF3395E0FE12674522A0
:1052B300900011E0FFEF3395E0FE12674522900066
:1052C30012E0FFEF3395E0FE12674522900013E0F2
:1052D300FFEF3395E0FE12674522900014E0FFEFE5
:1052E3003395E0FE12674522900015E0FFEF3395FA
:0552F300E0FE1267451A
:0152F8002293
:1064C3009001D6E4F0A3E4F09001DCE4F09001DC69
:1064D300E0FFD3EF64809483400302655F9001D8AB
:1064E300121FB1000186A020983E9001D8E0FCA3C2
:1064F300E0FDA3E0FEA3E0FFEC4D4E4F602A9001C8
:10650300D8E0FCA3E0FDA3E0FEA3E0FF7BFF7AFF5E
:1065130079FF78FFEF2BFFEE3AFEED39FDEC38FC07
:106523009001D8121FA580BFC2989001D6E0FEA3A8
:10653300E0FF7C007D0A121E47AD997C00EF2DFF22
:10654300EE3CFEEF24D0FFEE34FFFE9001D6EEF0DA
:10655300A3EFF09001DCE004F00264D09001D6E0F8
:04656300FEA3E0FFB4
:016567002211
:1052F9009001E5121FB1000186A020983E9001E5BA
:10530900E0FCA3E0FDA3E0FEA3E0FFEC4D4E4F60FF
:105319002A9001E5E0FCA3E0FDA3E0FEA3E0FF7B0A
:10532900FF7AFF79FF78FFEF2BFFEE3AFEED39FDAB
:10533900EC38FC9001E5121FA580BFC298AF99EF28
:10534900122002538C61539B6253AA6353B964536D
:10535900C86553D76653E66753F56854046954130F
:105369006A54226B54316C54406D544F74545575C2
:10537900546176546D7754797854857954917A00CB
:1053890000549C1264C3900022EEF0A3EFF0124D7A
:10539900F8221264C3900024EEF0A3EFF0124DF846
:1053A900221264C3900026EEF0A3EFF0124DF8220A
:1053B9001264C3900028EEF0A3EFF0124DF8221208
:1053C90064C390002AEEF0A3EFF0124DF8221264A4
:1053D900C390002CEEF0A3EFF0124DF8221264C333
:1053E90090002EEEF0A3EFF0124DF8221264C39054
:1053F9000030EEF0A3EFF0124DF8221264C39000D2
:1054090032EEF0A3EFF0124DF8221264C39000348B
:10541900EEF0A3EFF0124DF8221264C3900036EEBD
:10542900F0A3EFF0124DF8221264C3900038EEF0A9
:10543900A3EFF0124DF8221264C390003AEEF0A3E4
:10544900EFF0124DF822A217B39217221264C390FB
:105459000010EFF0124CF4221264C3900011EFF027
:10546900124CF4221264C3900012EFF0124CF42291
:105479001264C3900013EFF0124CF4221264C3902B
:105489000014EFF0124CF4221264C3900015EFF0EF
:03549900124CF4BE
:01549C0022ED
:1017F300021BB9E86480F8E933E83360110460F050
:10180300ED33EC337009E8FCE9FDEAFEEBFF22045B
:1018130060DED3EB9FEA9EE99DE8C2E78CF0C2F756
:1018230095F0400CE8CCF8E9CDF9EACEFAEBCFFB22
:10183300121B8485D0F05804700320D5B3E80470DC
:10184300075002B2D5021BC392D5EC0460F7E4CC77
:10185300C0E0C398F8603B94186008400DD0E0FBEB
:10186300021B9BE4FBFAC9FC8028E830E406E4C9C8
:10187300FBE4CAFCE830E305E4C9CACBFCE854073F
:101883006010F8C3E913F9EA13FAEB13FBEC13FC4A
:10189300D8F130F52FC3E49CFCEF9BFFEE9AFEEDED
:1018A30099FDD0E0FBEF4E4D4C701222DB03021B7F
:1018B300C0EC2CFCEF33FFEE33FEED33FDED30E7F0
:1018C300EB021B9BEF2BFFEE3AFEED39FDD0E0FB65
:1018D30050130BBB0003021BC3ED13FDEE13FEEF0E
:0818E30013FFEC13FC021B9B38
:1018EB00EC4D6011E8497017ED33EC3304600DE4F7
:1018FB00FCFFFEFD22E933E8330470F8021BB9123A
:10190B001B8458046009E4CC24815006285009023A
:10191B001BC3284003021BC0C0E0EB4A7044B980D4
:10192B0006D0E0FB021BAFEF4E701CBD8008EBFF37
:10193B00EAFEE9FD80EBE98DF0A4FEE5F00219D497
:10194B00E9CDF9EAFEEBFFEF89F0A4FCE5F0CE89D7
:10195B00F0A42EFFE435F0CD89F0A42DFEE435F094
:10196B008067EF4E7005BD80D780C3EF8BF0A4ACC2
:10197B00F0EE8BF0A42CFCE435F0F8EF8AF0A42CFD
:10198B00E5F038FCE433CB8DF0A42CFCE5F03BF810
:10199B00EE8AF0A42CFCE5F038F8E433CF89F0A400
:1019AB002CFCE5F038CF3400CE89F0A42FFFE5F006
:1019BB003EFEE433C98DF0A42EFEE5F039CD8AF05E
:1019CB00A42FFFE5F03EFEE43DFD33D0E0FB5007D6
:1019DB000BBB000F021BC3EC2CFCEF33FFEE33FEF3
:0619EB00ED33FD021B9B21
:1019F100021BC3EC5D046005E859047003021BB9C6
:101A0100121B84580460F6EC4860F2EC7004FDFE91
:101A1100FF22C860DB2481C85009C39860025006C8
:101A2100021BC09850CAF582E9294B4A7005AB8266
:101A3100021BAF75F0007C1A7880C3EF9BEE9AED24
:101A410099400DC3EF9BFFEE9AFEED99FDE842F040
:101A5100DC23ACF0D0E0FFD0E0FED0E0FDAB822093
:101A6100E7101BEB60BAEC2CFCEF33FFEE33FEED1D
:101A710033FD021B9BE803F830E705C0F075F00069
:101A8100EF2FFFEE33FEED33FD40B830E7C280AA01
:101A910074F8CC6480CCC86480C8F582046043C308
:101AA100EB9FF5F0EA9E42F0E99D42F0E89C45F09B
:101AB10060305018E5825FFFE582F42B5582FB50C0
:101AC100210ABA001D09B90019088016E5825BFBDD
:101AD100E582F42F5582FF50090EBE00050DBD00B1
:101AE100010CC3EB9FF5F0EA9E42F0E99D42F0E85C
:0D1AF1009C45F06007CC4820E701B3EC22D3
:101AFE00ED33EC33600A047003BD8004ECB2E7FCF6
:011B0E0022B4
:101B0F0075F020800E75F010800575F0087D007E51
:101B1F00007F003392D530D503121EF4EC33401002
:101B2F00EF33FFEE33FEED33FDEC33FCD5F0ED225A
:0E1B3F00E5F0247EA2D513CC92E7CDCEFF2296
:101B4D00EDD2E7CD33EC3392D524814006E4FFFE90
:101B5D00FDFC22FCE4CFCECDCC24E0501174FF80EF
:101B6D00EDC3CC13CCCD13CDCE13CECF13CF04708C
:071B7D00F030D5DE021EF47A
:10373A00E56F24DBF582E43400F583E0056F22901F
:10374A0000D83009039000DBE475F001121FE20291
:10375A001DEF2002E97F2ED2028018EF540F249029
:10376A00D43440D4FF30060BEF24BFB41A00500300
:10377A002461FFE570600215700573E57370020538
:10378A007230090E9000D8E475F001121FE2EF02C0
:10379A001E350269E07403D2098003E4C209F56F99
:1037AA009000D8121FF9E4F570F572F573E57060B0
:1037BA00077F2012377D80F57571FFC203C202C2EE
:1037CA0004C205C207C208C20A123749FF700D3087
:1037DA0009057F0012378EAF73AE7222B4255FC21D
:1037EA00D5C206123749FF24D0B40A00501A75F020
:1037FA000A787030D50508B6FF0106C6A426F62059
:10380A00D5047002D20580D924CFB41A00EF50042F
:10381A00C2E5D206023A80D20380C6D20280C0D262
:10382A000480BCD2D580BAD20780B47F2012377DFB
:10383A002004077401B5700040F112373AFF1237BD
:10384A007D0237B7D20AD208809512373AFB12376F
:10385A003AFA12373AF94A4B7006797E7A3B7BFF7D
:10386A0020042EE570602A7E008E82758300121E67
:10387A000860060EEE657170F0C2D5EBC0E0EAC0D2
:10388A00E0E9C0E0EE123AE1D0E0F9D0E0FAD0E0A7
:10389A00FB121DEFFF60AAEBC0E0EAC0E0E9C0E05E
:1038AA0012377DD0E02401F9D0E03400FAD0E0FBF1
:1038BA00E5710460DCD571D98087D20480A2123AFE
:1038CA00C360F7E571700104121BCEA971600DE5A2
:1038DA0071600914F571123B6BEF60F3EA30E7028D
:1038EA00F404C3995079EAF425710430E701E40439
:1038FA00F571800D123AC360C1EA05712571121B78
:10390A00CEEA900107F030E701E4257104D571048D
:10391A0020070114123AE1E4C0E0123B6B90010760
:10392A00E0601320E70714F0123765802204F0D014
:10393A00E014C0E07F00123765E571600712375C5A
:10394A001571800B30070312375CD0E00237B7D00D
:10395A00E00480C4123AC3609EE57104121BCE9043
:10396A000107EAF0E5712007026001042404123A13
:01397A00E16B
:10397B0074FF04C0E0123B6B123765E57120070240
:10398B00600312375CD0E0B571E87F4512376F905A
:10399B000107E07F2B30E7047F2DF404C0E01237E2
:1039AB007DD0E075F00A84C0F0123766D0E0123794
:1039BB00660237B7791080027908C208C20A8008FC
:1039CB00D2D5790A8004790AC2D5E571047002F563
:1039DB0071E4FAFDFEFF12373AFC7B082003131249
:1039EB00373AFD7B1030020A12373AFE12373AFF94
:1039FB007B20EC3382D592D55013C3E43002069F63
:103A0B00FFE49EFEE42003039DFDE49CFCE4CBF865
:103A1B00C203EC700CCFCECDCCE824F8F870F38059
:103A2B0017C3EF33FFEE33FEED33FDEC33FCEB331B
:103A3B00FB994002FB0FD8E9EB300305F8D0E0C44B
:103A4B0048B203C0E00AEC4D4E4F78207B0070C2A9
:103A5B00EAB5710040BCC0E0123AE3D0F0D0E020F0
:103A6B000304C4C0E0C4B203C0F0123766D0F0D573
:103A7B00F0EB0237B712200238545339BF583825B0
:103A8B004C38214239C34F39CB4439CB49383A43AF
:103A9B0039D15538FE46395E4538C8473B9E5038BC
:103AAB00292D382D2E38502B383123384E203B877B
:103ABB002A37E94800003848E571B4FF03757106F1
:103ACB0012373AFC12373AFD12373AFE12373AFFE9
:103ADB00900100021C0B790AA2D5200514300709AE
:103AEB00B910020404B9080104A2D5200802500140
:103AFB00042004689204B570005034C0E07F20307D
:103B0B0005197F30A20472087207500F123B3AC29C
:103B1B0004C208C207C20A7F30800F300703E9C016
:103B2B00E012377D300703D0E0F9D0E0B570CC3030
:103B3B0007177F30B9100C12377D7F583006077F7F
:103B4B00788003B9080312377D3004057F2D0237C7
:103B5B007D7F20200AF87F2B2008F322920480CF50
:103B6B007F00B40700500B2400F582E43401F58389
:103B7B00E0FF22286E756C6C2900D20312373A30A5
:103B8B0003F8C203787030D50108F60237E92D50DF
:103B9B0043495812373A2403B405004001E4903BE3
:103BAB00999312376E743A12376ED2057570040200
:023BBB0039BF10
:0D6A5200ED33EC3360065004EC6480FC2250
:10641700021BB922EDA2E7D2E7F9EC3340F260F3B1
:10642700B4FF08ED547F70E8021BC3F82481C2E073
:10643700C0E0F40428FAC313FCED92E7FD9000CC0A
:10644700121FA5EEA2E7E9BA7F02C3133400940036
:10645700FA75F091A4E5F013F494FE8AF0A433E5FD
:10646700F033248CD313FDE492E7FE7F007C3F7565
:106477008302ECC0E0F8EDC0E0F9EEC0E0FAEFC04F
:10648700E0FB8583F09000CC121F4D85F083121935
:10649700F4D0E0FBD0E0FAD0E0F9D0E0F81217FA38
:1064A700ED6480FD30E7011CD583C7ED33CC33F8AD
:0C64B700D0E0A2E71328C313CC13FD2291
:1066A8009000CC121FA59000D0E0F8A3E0F9A3E079
:1066B800FAA3E0FB9000CCE0FCA3E0FDA3E0FEA37E
:1066C800E0FF1219F41259EC9000CC121FA59000AB
:1066D800D0E030E7599000CCE0FCA3E0FDA3E0FE59
:1066E800A3E0FFECC0E0EDC0E0EEC0E0EFC0E0E406
:1066F800FFFEFDFC9000CCE0F8A3E0F9A3E0FAA3CC
:10670800E0FB121A917BDB600250087A0F79497816
:106718004080067A0F794978C0D0E0FFD0E0FED0FB
:10672800E0FDD0E0FC1217FA9000CC121FA59000F3
:0D673800CCE0FCA3E0FDA3E0FEA3E0FF2207
:10549D003A70FA83BCAAE9E43E81E0F8BF9DE9E6E3
:1054AD003F80000039283C1ABB9969663DA335E35E
:1054BD00BF255DE73FC90FDB418DDBCCC44936EE1F
:1054CD0045C9913FC5B0F83D3F800000C317F53485
:1054DD00452FFA73C60AFDDD1255A604A2E192000E
:1054ED001420E01590549D7404121D108030125537
:1054FD00A630E102B20020E0EBA883A9829000CC97
:10550D00121FA5898288839054B17404121D1085D1
:10551D0082F09000CC121F6985F0821218EBED4CD1
:10552D006007300004EC6480FC221255A6C0E0A890
:10553D0083A9829000CC121FA5898288839054D5AF
:10554D007403121D108582F09000CC121F6985F036
:10555D00821218EB9000CCE0CCF0A3E0CDF0A3E0EC
:10556D00CEF0A3E0CFF09054C57403121D10D0827D
:10557D008582F09000CC121F6985F082E58230E0C3
:10558D00071219F4B2008096EFCBFFEECAFEEDC9FB
:10559D00FDECC8FC1219F48085ED33EC547FCC334F
:1055AD00920024605007D0E0D0E0021BB97B837AD3
:1055BD00F97922783E1218EBEDF933ECF8332481AA
:1055CD005011EFFBEEFA121B4D121B0FECB2E7FC64
:1055DD001217FAED33EC33602F2403F8C313FCEDEF
:1055ED0092E7FDE82481E4501FECF8EDF9EEFAEFB7
:1055FD00FB121B4DEF04C2E0FCF582121B19ECB23D
:10560D00E7FC1217FAE58203FAED33EC3360071469
:08561D0013FCED92E7FDEA2207
:1059CC00BE1249253E4CCCCDBEAAAAAB3F800000EE
:1059DC003E7ADBB03EED63383F24BC7D3F490FDBA4
:1059EC00ED33ECC2E7CC339200B4FF13ED547F607F
:1059FC0003021BB97FDB7E0F7DC97C3F025AE1C2DB
:105A0C0001C3947F401E7007EDD2E794904015EFD0
:105A1C00FBEEFAEDF9ECF87F007E007D807C3F1206
:105A2C0019F4D201ED33EC33248430E705E4C0E003
:105A3C00806B04FAEDD2E754F0C333DAFD5407342B
:105A4C00002323C0E0CCC0E0F8EDC0E0F9EEC0E0EC
:105A5C00FAEFC0E0FBE4121B19EC24FEFC9000D41E
:105A6C00121FA51218EB7B007A007980783F121771
:105A7C00FA9000D4E0B2E7CCF0A3E0CDF0A3E0CEF6
:105A8C00F0A3E0CFF0D0E0FBD0E0FAD0E0F9D0E02A
:105A9C00F81217FA9000D4121F691219F49000D45E
:105AAC00121FA59059CC7403121D109000D4121F14
:105ABC00691218EBD0E0600F24D8F582E43459F564
:105ACC0083121F751217FA30010B7BDB7A0F79C921
:105ADC0078BF1217FAED33EC336006ECA20092E7B4
:025AEC00FC229A
:105E03009000CC121FA574FFFFFEFDFC9000CCE0B8
:105E1300F8A3E0F9A3E0FAA3E0FBC3121F02603882
:105E23007F807E967D187C4B9000CCE0F8A3E0F950
:105E3300A3E0FAA3E0FB121A916002501B7F807E5D
:105E4300967D187CCB9000CCE0F8A3E0F9A3E0FAB0
:105E5300A3E0FB121A91500F9000CCE0FCA3E0FDED
:105E6300A3E0FEA3E0FF229000CCE0FCA3E0FDA3AF
:105E7300E0FEA3E0FF121B4D9000D0121FA590007F
:105E8300D0E0FCA3E0FDA3E0FEA3E0FFEC121B0FB8
:105E9300C8ECC8C9EDC9CAEECACBEFCB9000CCE0C1
:105EA300FCA3E0FDA3E0FEA3E0FF1217F6E4FBFA78
:105EB300F9F8121A91602640249000D0E0FCA3E088
:105EC300FDA3E0FEA3E0FFEF24FFFFEE34FFFEEDB2
:105ED30034FFFDEC34FFFC9000D0121FA59000D0DE
:105EE300E0FCA3E0FDA3E0FEA3E0FFEC121B0F2206
:101B8400E9D2E7C933E833F892D5EDD2E7CD33ECA7
:071B940033FC5002B2D52220
:101B9B00EC30E7100FBF000C0EBE00080DBD0004AB
:101BAB000BEB6014A2D5EB13FCED92E7FD2274FF57
:101BBB00FCFDFEFF22E480F8A2D574FF13FC7D80B0
:031BCB00E480EFC4
:101BCE00F920E73624F950037907E4F42402FBE503
:101BDE0082158270021583DBF6E024FB501BE96050
:101BEE0014E4F0E582158270021583E004F0B40A65
:0D1BFE0008E4F0D9EE7401F00A22C2D522ED
:101C0B00ED33EC3392D5FA602AB4FF33EDC2E77BA8
:101C1B00FF60067A1C7930E4227A1C793920D504CE
:101C2B007A1C7934224E614E002B494E46002D49C9
:101C3B004E4600E47A08F0A3DAFC7B00740722C05E
:101C4B0083C082ECC0E0EDC0E0EEC0E0EFC0E0EAA4
:101C5B0075F010A4CAABF075F04DA42BFBE435F076
:101C6B00FCEA2410FAEB34C5FBEC34D9FCEDC2E7EB
:101C7B00FF75F056A4F42411C5F0F434C58FF0A40D
:101C8B002AE5F03BE43CF020E714121D8DD0E0FF79
:101C9B00D0E0FED0E0FDD0E0FC1219F48014F40487
:101CAB00121D8DD0E0FFD0E0FED0E0FDD0E0FC12A5
:101CBB0018EBD082D083E0FAEDD2E7CD33EC3324AE
:101CCB0082FBE4C3CF33CFCE33CECD33CD33DBF377
:101CDB007B0775F00A846004F0A31B0AE5F0F0A300
:101CEB008FF0740AA4FFACF08EF0740AA42CFEAC37
:101CFB00F050010C8DF0740AA42CFDE435F0F0A328
:051D0B00DBDE7407227D
:101D1000C0E0EFFBEEFAEDF9ECF81218EBD0E0F5CD
:101D2000F0EFFBEEFAEDF9ECF8121F59A3A3A3A311
:101D3000E8C0E0E9C0E0EAC0E0EBC0E0C0F01218A3
:101D4000EB121F75A3A3A3A31217FAD0F0D0E0FBE8
:0D1D5000D0E0FAD0E0F9D0E0F8D5F0D422D0
:101D5D003F8000004120000042C80000447A00008E
:101D6D00461C400047C35000497424004B18968010
:101D7D004CBEBC205A0E1BCA6753C21C749DC5AE07
:101D8D00FB60065407601C2323121DBBEB54386007
:101D9D0009121DA7121DB61218EBECF8EDF9EEFAAB
:101DAD00EFCB22EB121DB680F1543803241C901D8D
:101DBD005DFE93FC0EEE93FD0EEE930ECE93FF2281
:106628000221C2E493A3F8E493A34003F68001F2A5
:1066380008DFF48029E493A3F85407240CC8C33373
:10664800C4540F4420C8834004F456800146F6DF42
:10665800E4800B010204081020408090693FE47E2A
:10666800019360BCA3FF543F30E509541FFEE49337
:10667800A360010ECF54C025E060A840B8E493A3FE
:10668800FAE493A3F8E493A3C8C582C8CAC583CA29
:10669800F0A3C8C582C8CAC583CADFE9DEE780BEE1
:01697F000017
:101DCD00C2D530F707B2D563F0FF05F030E70CB29E
:101DDD00D5F4048463F0FF05F080018430D502F45E
:021DED000422CE
:101DEF00BB010689828A83E0225002E722BBFE02F2
:091DFF00E32289828A83E4932225
:101E0800BB010CE58229F582E5833AF583E022508F
:101E180006E92582F8E622BBFE06E92582F8E222D9
:0D1E2800E58229F582E5833AF583E49322F3
:101E3500BB010689828A83F0225002F722BBFE018C
:021E4500F32286
:101E4700EF8DF0A4A8F0CF8CF0A428CE8DF0A42EAF
:021E5700FE2269
:101E5900C2D5EC30E709B2D5E4C39DFDE49CFCEEA4
:101E690030E715B2D5E4C39FFFE49EFE122055C3A7
:101E7900E49DFDE49CFC800312205530D507C3E4A2
:061E89009FFFE49EFE2213
:101E8F00C5F0F8A3E028F0C5F0F8E58215827002DE
:061E9F001583E038F0227B
:101EA500E88FF0A4CC8BF0A42CFCE98EF0A42CFCDC
:101EB5008AF0EDA42CFCEA8EF0A4CDA8F08BF0A45A
:101EC5002DCC3825F0FDE98FF0A42CCD35F0FCEBB9
:101ED5008EF0A4FEA9F0EB8FF0A4CFC5F02ECD397E
:0F1EE500FEE43CFCEAA42DCE35F0FDE43CFC22EB
:1068B900C2D5E830E70FB2D5E4C39BFBE49AFAE40A
:1068C90099F9E498F8EC30E717B2D51268EF12207D
:1068D900E6E4C39BFBE49AFAE499F9E498F88003A7
:1068E9001220E630D50DE4C39FFFE49EFEE49DFD32
:0468F900E49CFC22FD
:0E1EF400C3E49FFFE49EFEE49DFDE49CFC22FF
:101F0200EB9FF5F0EA9E42F0E99D42F0E89C45F035
:011F120022AC
:101F1300BB010789828A83021F4D5005E9F802211C
:101F230078BBFE05E9F802218489828A83021F595E
:101F3300BB010789828A83021FA55005E9F80221A4
:0A1F4300AABBFE05E9F80221B62250
:0C1F4D00E0FCA3E0FDA3E0FEA3E0FF2207
:101F5900E493FC740193FD740293FE740393FF22CE
:0C1F6900E0F8A3E0F9A3E0FAA3E0FB22FB
:101F7500E493F8740193F9740293FA740393FB22C2
:101F8500BB010789828A83021F695005E9F802218E
:101F950090BBFE05E9F802219D89828A83021F759F
:0C1FA500ECF0A3EDF0A3EEF0A3EFF022AF
:101FB100A8828583F0D083D082121FC8121FC81255
:101FC1001FC8121FC8E473E493A3C583C5F0C5837A
:101FD100C8C582C8F0A3C583C5F0C583C8C582C87A
:011FE10022DD
:101FE200F8E0FBA3A3E0F925F0F0E5821582700288
:071FF2001583E0FA38F0222C
:091FF900EBF0A3EAF0A3E9F022E9
:10200200D083D082F8E4937012740193700DA3A36D
:1020120093F8740193F5828883E473740293686081
:06202200EFA3A3A380DF81
:10202800D083D082F8E4937012740193700DA3A347
:1020380093F8740193F5828883E473740293B5F07E
:0D204800067403936860E9A3A3A3A380D8E6
:1069E000EFB40A07740D1269EB740A309811A89974
:1069F000B8130CC2983098FDA899C298B811F63017
:076A000099FDC299F59922EE
:10000E00C3EE6480948040028007C3E49FFFE49EA9
:02001E00FE22C0
:10205500BC000BBE0029EF8DF084FFADF022E4CC6F
:10206500F875F008EF2FFFEE33FEEC33FCEE9DEC38
:10207500984005FCEE9DFE0FD5F0E9E4CEFD22ED7E
:10208500F8F5F0EE8420D21CFEADF075F008EF2FC8
:10209500FFED33FD4007985006D5F0F222C398FDB9
:0520A5000FD5F0EA2256
:1020AA0075F008758200EF2FFFEE33FECD33CDCCED
:1020BA0033CCC58233C5829BED9AEC99E582984070
:1020CA000CF582EE9BFEED9AFDEC99FC0FD5F0D64D
:1020DA00E4CEFBE4CDFAE4CCF9A88222B800C1B977
:1020EA000059BA002DEC8BF084CFCECDFCE5F0CBB5
:1020FA00F97818EF2FFFEE33FEED33FDEC33FCEBEE
:10210A0033FB10D703994004EB99FB0FD8E5E4F9A8
:10211A00FA227818EF2FFFEE33FEED33FDEC33FC95
:10212A00C933C910D7059BE99A4007EC9BFCE99A89
:10213A00F90FD8E0E4C9FAE4CCFB2275F010EF2FCE
:10214A00FFEE33FEED33FDCC33CCC833C810D707CE
:10215A009BEC9AE899400AED9BFDEC9AFCE899F809
:0E216A000FD5F0DAE4CDFBE4CCFAE4C8F9229C
:0C217800E6FC08E6FD08E6FE08E6FF2293
:0C218400E2FC08E2FD08E2FE08E2FF2297
:0D219000E6FB08E6F908E6FA08E6CBF822BF
:0D219D00E2FB08E2F908E2FA08E2CBF822C2
:0C21AA00ECF608EDF608EEF608EFF62261
:0C21B600ECF208EDF208EEF208EFF22265
:00000001FF
